:1000000000400020E15C0000215D0000235D000055
:1000100000000000000000000000000000000000E0
:10002000000000000000000000000000255D00004E
:100030000000000000000000275D0000295D0000B6
:100040002B5D00002B5D0000056100002B5D0000B2
:100050002B5D0000000000002B5D00002B5D000008
:100060002B5D0000DD6300002B5D00002B5D0000B8
:100070002B5D00002B5D00002B5D00002B5D000060
:100080002B5D0000416500002B5D00002B5D000032
:100090002B5D00002B5D00002B5D00002B5D000040
:1000A0002B5D00002B5D0000000000000000000040
:1000B0000000000000000000000000000000000040
:1000C000054B0648033310B51B1A062B03D9044B06
:1000D000002B00D0984710BDA0020020A0020020F5
:1000E000000000000648074910B5091A8910CB0F17
:1000F0005918491003D0044B002B00D0984710BD6D
:10010000A0020020A00200200000000010B5074C53
:100110002378002B09D1FFF7D3FF054B002B02D02A
:10012000044800E000BF0123237010BDA00200209E
:1001300000000000C8A80000094B10B5002B03D038
:100140000849094800E000BF08480368002B02D1B5
:10015000FFF7C8FF10BD064B002BF9D09847F7E713
:1001600000000000A4020020C8A800009C0200209B
:1001700000000000164B002B00D1144B9D4640227E
:1001800092029A1A924600218B460F461348144A4F
:10019000121A08F0B4F80F4B002B00D098470E4B02
:1001A000002B00D098470020002104000D000D48CE
:1001B000002802D00C4800E000BF08F05DF82000E5
:1001C000290005F0B7FF08F031F8C046000008002C
:1001D000004000200000000000000000A0020020FD
:1001E000E42500200000000000000000012303407F
:1001F0000200181E04D1042A03D91068000900E087
:100200000020704710B50400FFF7F0FF0300002046
:1002100083420BD0013B9B00181DE2181279002A83
:1002200003D001338342F8D100E0180010BD012251
:10023000096810B5114201D0002903DA102000F03E
:1002400083F903E04910062002F09CF810BD09680C
:1002500010B5CB0701D5002903DA102000F074F99E
:1002600006E04910033189100022052002F08AF8C7
:1002700010BD70B50D68AB0728D1042D26D90F230A
:100280002A684E681340062B09D12800FFF7AEFFFD
:10029000012383421DDC9A00AE500133F9E7052BA0
:1002A00014D1F30703D4132000F04EF912E07610B6
:1002B000FF2EF8D82800FFF799FF2C1D230080009F
:1002C0002018984205D91E700133FAE70B2000F080
:1002D0003BF9002070BD70B50C681120E3072DD5E7
:1002E0004D68AB0729D1042D27D90F262B68641040
:1002F0001E40062E0BD1002C04DD2800FFF776FFF0
:10030000844201DD122019E0A400605918E0331F77
:10031000012B12D82800FFF769FF8000042E02D1BC
:100320002800FFF76FFF002CECDDA042EADB012381
:100330002C19E0784000184302E00B2000F004F98B
:1003400070BDF8B501230C6811201C422FD0032585
:100350004E6835402AD1042E28D90F233268641004
:100360008F681340062B0BD1002C04DD3000FFF703
:100370003DFF844201DD122019E0A400A75113E0E3
:10038000052B13D1002CF6DD3000FFF72FFF800086
:100390008442F0DC01231F4201D1132007E07F10CB
:1003A000FF2FFAD83419E770280002E00B2000F084
:1003B000CBF8F8BD086810B5830717D1042815D904
:1003C0000F2302681340062B02D1FFF70FFF0BE04B
:1003D000052B05D1FFF70AFFC0000123184308E0F1
:1003E000042B03D1FFF70EFF4000F6E70B2000F0CF
:1003F000ABF810BD012303400200181E01D05010BD
:1004000002E00D22014B1A707047C046BC0200206A
:10041000012303400200181E04D1042A03D91068E6
:10042000000900E00020704770B50D000400FFF7E0
:10043000EFFF86002800FFF7EBFF830000209E42BD
:100440000ED1231D9E1904351A009E4207D9297822
:100450001278013301358A42F6D0002000E00120F5
:1004600070BD0000F0B585B00393019002912D4E50
:100470002D4B002A02D002223270013A00251A6068
:100480001B68F554019B9D424ADA029AAB00D05892
:10049000254B1C68C8239B0037191C1B01231842DD
:1004A00002D04310214A1FE0214A002802D004282C
:1004B00005D1204A2100380008F0E8FA18E00428A5
:1004C00010D90F2302681340042B04D101F096FFCA
:1004D000194A030008E0062B05D1FFF799FF174AD8
:1004E000030001E00123164A2100380008F0CEFA8B
:1004F000300008F031FB039B0B4A002B01D1106048
:100500000CE0019B013B9D42F9DA0E4B9842F6DC70
:10051000431C1360202232540022F2540135B1E70B
:1005200005B0F0BDC8020020C40200207D98000084
:10053000509800005698000049A200005B98000007
:100540006C9800001F030000014B187000207047DA
:10055000BC02002070B501F071FD094C0100251DA1
:100560001F22280008F0FFFA280008F0F5FA0423FB
:1005700004308008000118432060200070BDC04690
:10058000E8050020C368F0B59D00836889B05D1957
:10059000030018330693036903909E00069B9F197E
:1005A00043699E000193069B9E19D54B1B78002B37
:1005B0000FD17F222B68D3491C1213409B005B583C
:1005C00001960435029235E0CD4B1B78002B29D0E3
:1005D000019E039BCA4C9B6821780193EA1A039BF6
:1005E00092109B7812021A43039B587803F02AFB5F
:1005F0000023039A2370137001960497039B069AB5
:100600009B68ED1A0293039BAD10DD60049B9F1A5B
:10061000039BBF101F61019B9B1A039A9B105361A0
:1006200001F086FC2B68029A1C121340B54A9B000D
:100630009B5804359F46039B587803F0FBFA002330
:10064000039A1370D9E7069B3A1DD11AAC4BDB29EC
:1006500003DD1A22019E1A70BBE71B783C60002B59
:1006600002D0019E1700B4E72B6802991C120B40C0
:10067000A4499B005B5817000435DBE7069B3A1D35
:10068000D11A9F4BDB2903DD1A22019E1A70A0E7C5
:1006900028681B78291D3860002B03D0019E1700A5
:1006A0000D0096E76B6802991C120B4095499B0060
:1006B0005B5817000835BDE7069B3A1DD11A904BD1
:1006C000DB2903DD1A22019E1A7082E7A4001B7841
:1006D0002C193C60002B02D0019E170079E72B6893
:1006E00002991C120B4087499B005B581700043588
:1006F000A0E7069B3A1DD11A814BDB2903DD1A22A4
:10070000019E1A7065E78048A40021581B78396063
:10071000002B02D0019E17005BE72B6802991C1288
:100720000B4078499B005B581700043582E7043F73
:10073000754B3A68A400E250714B1B78002B01D036
:10074000019E46E72B68029A1C1213406D4A9B00DB
:100750009B5804356EE76C4BA600F058FFF74AFE35
:10076000043F04003868FFF745FE24180120664B5B
:1007700064000443F450624B1B78002B01D0019EAF
:1007800027E72B68029A1C1213405E4A9B009B5875
:1007900004354FE7069B3A1DD11A594BDB2903DD7F
:1007A0001A22019E1A7014E70198069C0121A042AA
:1007B00002D901000C3909681B783960002B02D07E
:1007C000019E170005E72B6802991C120B404D494A
:1007D0009B005B58170004352CE7069B3A1DD11A85
:1007E000474BDB2903DD1A22019E1A70F1E60199BD
:1007F000069881420AD90B000C3B1B6843495B10E9
:100800006418E41A019BA400E35802E0182119704F
:1008100000233B603A4B1B78002B02D0019E17004F
:10082000D7E62B6802991C120B4036499B005B5897
:1008300017000435FEE6019B069A93420CD90C3B47
:100840001968324B3E1FE3184910591A3268019B50
:100850008900CA50370002E01822294B1A70284B31
:100860001B78002B01D0019EB3E62B68029A1C1264
:100870001340244A9B009B580435DBE6019B069AF3
:10088000934220D9214B3E1FE318019C04930C3C5A
:100890002368049A5B10D31A019A9B009858FFF7BB
:1008A000A9FD07903068FFF7A5FD2468049B64103C
:1008B0001C1B079BA4001F1801207F00019B0743FE
:1008C000E750370002E018220D4B1A700C4B1B78D2
:1008D000002B01D0019E7CE62B68029A1C1213406B
:1008E000084A9B009B580435A4E6069B3A1DD11A82
:1008F000034BDB290CDD1A22019E1A7069E6C04603
:10090000BC0200209098000028230020FDFFFF3F3C
:100910000199A40061581B783960002B02D0019E18
:10092000170056E62B6802991C120B40D0499B0019
:100930005B58170004357DE6043F019B3A68A4002C
:10094000E250CC4B1B78002B01D0019E41E62B6876
:10095000029A1C121340C64A9B009B58043569E654
:10096000019BA4001C192368043F38685E10FFF740
:1009700041FD36180120BF4B76001B7806432660E8
:10098000002B01D0019E24E62B68029A1C12134012
:10099000B74A9B009B5804354CE6069BA4003F1BBE
:1009A000B44CBB420DD82378002B01D0019E10E639
:1009B0002B68029A1C121340AD4A9B009B580435C9
:1009C00038E6AD4801F08EFC2378002B01D0019E63
:1009D000FFE52B68029A1C121340A54A9B009B5806
:1009E000043527E6A300ED18002C00DA05E6A14B3C
:1009F0001B78002B01D0019EEBE52B68029A1C129C
:100A000013409B4A9B009B58043513E63B1F0493FD
:100A10001B680793042B04D1A300ED18002C00DA07
:100A2000ECE5944B1B78002B02D0019E049FD0E58F
:100A30002B68029A1C1213408D4A9B009B58049FFE
:100A40000435F7E53B1F04931B68042B06D0A20076
:100A5000AD18002C02DA002B00D1CFE5854B1B78B6
:100A6000002B02D0019E049FB3E52B68029A1C1252
:100A700013407F4A9B009B58049F0435DAE53A1FD8
:100A800013685B10013B002B07DD01215B00A40014
:100A90000B4304972D191360B0E5764B17001B78B4
:100AA000002B01D0019E94E52B68029A1C12134082
:100AB0006F4A9B009B580435BCE53A00069B0C32FC
:100AC000D31ADB2B04DD1A226A4B019E1A7080E5D3
:100AD000FF2361005B000B4001210B433B60039B44
:100AE00006989B6824120493ED1A039BAD109B7823
:100AF0002D021D43019B8D401B1A9B108B400B4305
:100B0000BB60039B0D437D609C70E4B25B4BE400D3
:100B10000399E35816008B6056490978002903D0E1
:100B200008331D00170054E51D0002999B680C3521
:100B30001C120B404E499B005B580192170079E54F
:100B40003B1F1C68069A019B93422AD104970A20F6
:100B5000E30716D4A3070DD1042C0BD90F23226869
:100B60001340042B06D1200001F048FC07F0F4FFED
:100B7000063006E00720042C03D0002C01D0802092
:100B80008000643002F004FE002801D1043D35E508
:100B9000039B2100587803F067F80023039A137031
:100BA0002CE5019B019A0C3B1B6803995B109B0091
:100BB0005B421E00D3180C3B1C601300083B1B68F3
:100BC000083E97195A108A70D2B22C49D2005B00A5
:100BD00055589B0A039A9B009560ED18019B043BB6
:100BE0001E68069B7610B6009E19224B1B78002BC0
:100BF00000D0EEE42B68029A1C1213401C4A9B00A2
:100C00009B580196043515E53B1F1868FFF7F2FB6A
:100C1000A40006003F1B1E2834DC00280EDC154B08
:100C20001B78002B01D0019ED3E42B68029A1C1282
:100C300013400F4A9B009B580435FBE401F0E4F994
:100C4000033E361801F0E0F90D4B801B9842F9D8AD
:100C5000084B1B78002B01D0019EBAE42B68029A46
:100C60001C121340024A9B009B580435E2E4C04624
:100C700090980000BC02002080980000301B0020EB
:100C80009F8601000123039A137001F0BDF9039BB5
:100C90000A3886195E60B0E43B1F1868FFF7AAFBAC
:100CA000A40004903F1B00280EDCCA4B1B78002BCD
:100CB00001D0019E8DE42B68029A1C121340C64A93
:100CC0009B009B580435B5E4C44B049A019E9A429C
:100CD00003DD1D22BF4B1A707BE40123039A1370BE
:100CE00001F092F9FA23049A9B005343039A0A3BBA
:100CF0001B18536081E4A300FF1A002320001A0090
:100D00003900FFF7AFFBB64EB64C3168200002F059
:100D1000FBFE3168200002F0AEFF3168200001F0D8
:100D200043FCAC4B1B78002B01D0019E51E42B6897
:100D3000029A1C121340A84A9B009B58043579E480
:100D4000A44BA4001B783F1B002B01D0019E40E464
:100D50002B68029A1C1213409F4A9B009B58043533
:100D600068E402F05BFD01F0E3F83B1F186800281F
:100D700023D1083B1868C30701D5401016E083074C
:100D80000FD104280DD90F2302681340062B02D17E
:100D9000FFF73EFB0AE0052B03D1FFF739FB80008C
:100DA00004E019228B4B019E1A7012E43A000121D3
:100DB0004300083A0B43136001E04010013800285B
:100DC00032DD012243001343391F0B603B00083B17
:100DD0001B681341181A3B000C3B1B68134203D0DD
:100DE0008018A400904015E0990717D1042B15D95D
:100DF0000F211E683140062906D101308000C358FA
:100E0000019AA400A35010E0052907D11818007911
:100E1000A4004000019B1043E05006E019226D4BF6
:100E2000019E1A70FFF7D5FB04356A4B1B78002B27
:100E300002D0019EFFF7CDFB2B68029A1C121340D3
:100E4000654A9B009B580435FFF7F4FBA300069A04
:100E5000FB189B1ADB2B01DC012205E01A225D4BFB
:100E6000019E1A70FFF7B5FB631E002C03DD3A608C
:100E70001C000437F8E7574B1B78002B02D0019E6B
:100E8000FFF7A7FB2B68029A1C121340524A9B00E3
:100E90009B580435FFF7CEFB069A3B1D9B1A4D4E1F
:100EA000DB2B04DD1A233370019EFFF792FB019BBD
:100EB000069AA400934218D93B1F1868FFF79AFAC4
:100EC000002810DD019B0C3B1B685B1098420ADC7C
:100ED0009A07D31A1818444BC018019B8000C258B7
:100EE0003B1B1A6003E0202300E018233370394BCA
:100EF0003E1B1B78371D002B02D0019EFFF769FBBC
:100F00002B68029A1C121340334A9B009B580435ED
:100F1000FFF790FBA3009C46F81A002C04DC1C226F
:100F20002C4B00261A7015E0002103685B10012687
:100F30008A008258164003D10D22264B1A7009E010
:100F40005210934200DD130001318C42EFDC012688
:100F50005B001E4363460660FE1A1E4B371D1B785E
:100F6000002B02D0019EFFF734FB2B68029A1C1263
:100F70001340194A9B009B580435FFF75BFBA30005
:100F80009C46F81A002C04DC1C22124B00261A7016
:100F900015E0002103685B1001268A008258164084
:100FA00003D10D220B4B1A7009E05210934200DA64
:100FB000130001318C42EFDC01265B001E436346C7
:100FC0000660FE1A034B371D1B78002B0ED0019EC6
:100FD000FFF7FFFABC0200209098000080EE360078
:100FE000C4020020C8020020FCFFFF3F2B68029AC9
:100FF0001C121340D84A9B009B580435FFF71AFB7C
:101000003B00083B1868FFF7F5F93B1F0490186890
:10101000FFF7F0F9049AA600BC1B0023824200DA15
:1010200004332360CD4BBE1B1B78371D002B02D031
:10103000019EFFF7CEFA2B68029A1C121340C64A93
:101040009B009B580435FFF7F5FAA300FE1A0493A2
:101050003B00083B1868FFF7CDF93B1F04001868F8
:10106000FFF7C8F9E20FC317A04253419B0033605A
:10107000049BFE1AB94B371D1B78002B02D0019E32
:10108000FFF7A7FA2B68029A1C121340B24A9B0082
:101090009B580435FFF7CEFA3B00083B18683B1F0E
:1010A0001968A300884202D1FB1A042222E0042816
:1010B0001ED90122104201D0114219D1032630421B
:1010C00015D10F2302681A40042A10D131420ED1E3
:1010D00004290CD90A681340042B08D1FFF7A4F99E
:1010E000431E9841A600BE1B8000306003E0A300B1
:1010F0000022FB1A1A60994BA4001B783E1B371D77
:10110000002B02D0019EFFF764FA2B68029A1C1292
:101110001340914A9B009B580435FFF78BFA3B0024
:10112000083B18683B1F1968A300884202D1FB1ACC
:10113000002223E004281FD90122104201D01142CD
:101140001AD10326304216D10F2302681A40042A0E
:1011500011D131420FD104290DD90A681340042B53
:1011600009D1FFF761F9030058425841A600BE1BA0
:101170008000306003E0A3000422FB1A1A60774B62
:10118000A4001B783E1B371D002B02D0019EFFF7E9
:1011900020FA2B68029A1C1213406F4A9B009B583E
:1011A0000435FFF747FAA300FE1A04933B00083BFF
:1011B0001868FFF71FF93B1F04001868FFF71AF9BA
:1011C000E217C30F844253419B003360049BFE1A15
:1011D000624B371D1B78002B02D0019EFFF7F9F9F7
:1011E0002B68029A1C1213405B4A9B009B580435E3
:1011F000FFF720FA3B00083B1868FFF7FBF83B1F9E
:1012000004901868FFF7F6F8049AA600BC1B0023A8
:10121000824200DD04332360504BBE1B1B78371D18
:10122000002B02D0019EFFF7D4F92B68029A1C1202
:101230001340494A9B009B580435FFF7FBF93B1FBD
:101240001B68A400043B591E8B413A1B9B00136092
:10125000424B171D1B78002B02D0019EFFF7B9F9F6
:101260002B68029A1C1213403B4A9B009B58043582
:10127000FFF7E0F9A300FC1A04933B00083B186851
:10128000FFF7B8F83B1F06001868FFF7B3F83618E9
:101290000120049B760006432660FE1A2F4B371D63
:1012A0001B78002B02D0019EFFF793F92B68029A5E
:1012B0001C121340284A9B009B580435FFF7BAF9CB
:1012C000A300FE1A04933B00083B1868FFF792F84E
:1012D0003B1F04001868FFF78DF8241A0120049BB7
:1012E000640004433460FE1A1C4B371D1B78002B2E
:1012F00002D0019EFFF76DF92B68029A1C12134071
:10130000154A9B009B580435FFF794F9A300FC1A7B
:1013100004933B00083B1868FFF76CF83B1F06007E
:101320001868FFF767F846430120049B76000643E0
:101330002660FE1A094B371D1B78002B02D0019E38
:10134000FFF747F92B68029A1C121340024A9B00D0
:101350009B580435FFF76EF990980000BC020020FE
:101360003B1F1868FFF746F8A30006000493FC1A19
:10137000002803D11F22E84B1A700AE03B00083B0B
:101380001868FFF737F8310005F07EF901264000B4
:101390000643049B2660FE1ADF4B371D1B78002B8B
:1013A00002D0019EFFF715F92B68029A1C12134018
:1013B000DA4A9B009B580435FFF73CF93B1F18683D
:1013C000FFF718F8A30006000493FC1A002803D1C5
:1013D0001F22D14B1A700AE03B00083B1868FFF748
:1013E00009F8310005F036FA012649000E43049B46
:1013F0002660FE1AC84B371D1B78002B02D0019EB9
:10140000FFF7E7F82B68029A1C121340C34A9B00AF
:101410009B580435FFF70EF93B1F1868FEF7EAFFEB
:10142000C317C0185840012340001843BA4BA4000A
:101430001B783E1B3060371D002B02D0019EFFF74A
:10144000C8F82B68029A1C121340B44A9B009B58A0
:101450000435FFF7EFF8A300FE1A07933068012C5C
:1014600003D1FEF7C7FF049008E0FEF7C3FF0400B6
:101470007068FEF7BFFF0130031B0493049B002B31
:1014800001DC0123049307F0B3FA049905F0E2F9B3
:101490000C190121079B64000C433460FE1A9E4B1B
:1014A000371D1B78002B02D0019EFFF792F82B68A6
:1014B000029A1C121340994A9B009B580435FFF76F
:1014C000B9F8A300FE1A31002000049300F0A8FF31
:1014D000049B3060FE1A904B371D1B78002B02D006
:1014E000019EFFF776F82B68029A1C1213408B4A74
:1014F0009B009B580435FFF79DF8A300FE1A049348
:101500003B00083B1868FEF775FF3B1F0400186896
:10151000FEF770FF04400120049B64000443346024
:10152000FE1A7D4B371D1B78002B02D0019EFFF762
:1015300050F82B68029A1C121340784A9B009B5863
:101540000435FFF777F8A300FC1A04933B00083B2F
:101550001868FEF74FFF3B1F06001868FEF74AFFAA
:1015600006430120049B760006432660FE1A6A4B60
:10157000371D1B78002B02D0019EFFF72AF82B683D
:10158000029A1C121340654A9B009B580435FFF7D2
:1015900051F8A300FC1A04933B00083B1868FEF7BF
:1015A00029FF3B1F06001868FEF724FF4640012074
:1015B000049B760006432660FE1A574B371D1B78A6
:1015C000002B02D0019EFFF704F82B68029A1C1230
:1015D0001340524A9B009B580435FFF72BF83B1FE2
:1015E0001868FEF707FFC0430123400018434A4B29
:1015F000A4001B783E1B3060371D002B02D0019EDB
:10160000FEF7E7FF2B68029A1C121340434A9B0027
:101610009B580435FFF70EF8A300FE1A04933B0015
:10162000083B1868FEF7E6FE3B1F04001868FEF74B
:10163000E1FE8440012364001C43049B3460FE1AD5
:10164000354B371D1B78002B02D0019EFEF7C1FFE2
:101650002B68029A1C121340304A9B009B58043599
:10166000FEF7E8FFA300FE1A04933B00083B18684E
:10167000FEF7C0FE3B1F04001868FEF7BBFE0441E6
:10168000012364001C43049B3460FE1A224B371D67
:101690001B78002B02D0019EFEF79BFF2B68029A5D
:1016A0001C1213401D4A9B009B580435FEF7C2FFD5
:1016B0003B000C3B1868FEF79DFE3B00083B060014
:1016C0001868FEF797FEF1170200C317300005F007
:1016D00013F93B1F049005911868FEF78BFE02007A
:1016E0000498059905F0BCF80123400018430A4B03
:1016F000A4001B783E1B3060371D002B02D0019EDA
:10170000FEF767FF2B68029A1C121340034A9B00E6
:101710009B580435FEF78EFFBC0200209098000015
:10172000A300FE1A310020000493FEF780FD049B05
:101730003060FE1AE54B371D1B78002B02D0019E4E
:10174000FEF747FF2B68029A1C121340E04A9B00E9
:101750009B580435FEF76EFFA300FE1A31002000EF
:101760000493FEF774FD049B3060FE1AD74B371DBF
:101770001B78002B02D0019EFEF72BFF2B68029AEC
:101780001C121340D24A9B009B580435FEF752FFAF
:10179000A300FF1A39002000FEF76BFDCB4B1B782E
:1017A000002B02D0019EFEF714FF2B68029A1C1238
:1017B0001340C74A9B009B580435FEF73BFFA3002C
:1017C000FE1A310020000493FEF785FD049B306073
:1017D000FE1ABE4B371D1B78002B02D0019EFEF770
:1017E000F8FE2B68029A1C121340B94A9B009B58C2
:1017F0000435FEF71FFFA300FF1A39002000FEF793
:10180000A0FDB24B1B78002B02D0019EFEF7E1FE3B
:101810002B68029A1C121340AD4A9B009B5804355A
:10182000FEF708FFA300FE1A310020000493FEF724
:10183000C1FD049B3060FE1AA44B371D1B78002BA2
:1018400002D0019EFEF7C5FE2B68029A1C121340BF
:101850009F4A9B009B580435FEF7ECFE069A3B1D01
:1018600004939A4C9B1ADB2B04DD1A23019E2370F0
:10187000FEF7AFFE00F0D2FB0123400018432378AF
:101880003860002B03D0019E049FFEF7A2FE2B6858
:10189000029A1C1213408E4A9B009B58049F0435E9
:1018A000FEF7C8FE069A3B1D0493884C9B1ADB2B5F
:1018B00004DD1A23019E2370FEF78BFE00F0A4FBCB
:1018C000844B400018400123184323783860002BD4
:1018D00003D0019E049FFEF77CFE2B68029A1C1227
:1018E00013407B4A9B009B58049F0435FEF7A2FEE1
:1018F000A300FB1A0493012320001A000499FEF7A9
:10190000B1FD754C2068643001F042FF002816D00C
:10191000039B21685A78714802F0BBF915E0A300D7
:10192000FB1A04932000012300220499FEF79AFD7C
:10193000694C2068643001F02BFF002802D1043D7F
:10194000FEF75BFE654802F03DF80123039A137031
:1019500000F05AFB624A2368126806335343181892
:10196000039B5860FEF74AFEFEF7F4FD574BA400B8
:101970001B783E1B3060371D002B02D0019EFEF706
:1019800028FE2B68029A1C121340514A9B009B5858
:101990000435FEF74FFEA4003E1B300000F072FB42
:1019A0004A4B30601B78371D002B02D0019EFEF79A
:1019B00010FE2B68029A1C121340454A9B009B584C
:1019C0000435FEF737FEA4003E1B300000F05CFB40
:1019D0003E4B30601B78371D002B02D0019EFEF776
:1019E000F8FD2B68029A1C121340394A9B009B5841
:1019F0000435FEF71FFEA4003E1B300000F046FB3E
:101A0000324B30601B78371D002B02D0019EFEF751
:101A1000E0FD2B68029A1C1213402D4A9B009B5834
:101A20000435FEF707FEA4003F1B380000F04CFB16
:101A3000264B1B78002B02D0019EFEF7CAFD2B68B7
:101A4000029A1C121340224A9B009B580435FEF751
:101A5000F1FDA300FE1A31002000049300F056FBB4
:101A6000049B3060FE1A194B371D1B78002B02D0E7
:101A7000019EFEF7AEFD2B68029A1C121340144A19
:101A80009B009B580435FEF7D5FDA4003F1B380092
:101A900000F076FB0D4B1B78002B02D0019EFEF769
:101AA00098FD2B68029A1C121340094A9B009B5810
:101AB0000435FEF7BFFD0121200000F049FB034B78
:101AC0001B78002B0ED0019EFEF783FDBC02002088
:101AD00090980000FEFFFF7FC4020020C802002093
:101AE000040000202B68029A1C121340E94A9B0054
:101AF0009B580435FEF79EFD0021200000F028FBD6
:101B0000E54B1B78002B02D0019EFEF762FD2B688F
:101B1000029A1C121340DF4A9B009B580435FEF7C3
:101B200089FDA4003E1B300000F048FBDA4B30601A
:101B30001B78371D002B02D0019EFEF74AFD2B6853
:101B4000029A1C121340D34A9B009B580435FEF79F
:101B500071FDA4003E1B300000F044FBCE4B306012
:101B60001B78371D002B02D0019EFEF732FD2B683B
:101B7000029A1C121340C74A9B009B580435FEF77B
:101B800059FDA4003F1B380000F006FBC24B1B7838
:101B9000002B02D0019EFEF71CFD2B68029A1C123E
:101BA0001340BC4A9B009B580435FEF743FDA4003C
:101BB0003F1B380002F0E4FAB74B1B78002B02D031
:101BC000019EFEF706FD2B68029A1C121340B14AD3
:101BD0009B009B580435FEF72DFDA4003E1B3000F2
:101BE00002F078FBAC4B30601B78371D002B02D025
:101BF000019EFEF7EEFC2B68029A1C121340A54AC8
:101C00009B009B580435FEF715FDA4003F1B3800D0
:101C100002F086FAA04B1B78002B02D0019EFEF743
:101C2000D8FC2B68029A1C1213409A4A9B009B58BE
:101C30000435FEF7FFFCA4003E1B300002F086FADC
:101C4000954B30601B78371D002B02D0019EFEF7AC
:101C5000C0FC2B68029A1C1213408E4A9B009B58B2
:101C60000435FEF7E7FCA300FF1A3900200000F05E
:101C700003FF894B1B78002B02D0019EFEF7A9FCC5
:101C80002B68029A1C121340824A9B009B58043511
:101C9000FEF7D0FCA300FF1A3900200000F0B6FDCB
:101CA0007D4B1B78002B02D0019EFEF792FC2B6827
:101CB000029A1C121340774A9B009B580435FEF78A
:101CC000B9FCA300FF1A3900200000F0AFFD724BF1
:101CD0001B78002B02D0019EFEF77BFC2B68029A3A
:101CE0001C1213406B4A9B009B580435FEF7A2FC64
:101CF000A300FF1A3900200000F0C0FD664B1B78DE
:101D0000002B02D0019EFEF764FC2B68029A1C1285
:101D10001340604A9B009B580435FEF78BFCA300E0
:101D2000FE1A31002000049302F015FB049B306082
:101D3000FE1A594B371D1B78002B02D0019EFEF76F
:101D400048FC2B68029A1C121340524A9B009B5875
:101D50000435FEF76FFCA300FE1A31002000049347
:101D600002F011FB049B3060FE1A4B4B371D1B78B1
:101D7000002B02D0019EFEF72CFC2B68029A1C124D
:101D80001340444A9B009B580435FEF753FCA300C4
:101D9000FE1A31002000049302F0B7FA049B306071
:101DA000FE1A3D4B371D1B78002B02D0019EFEF71B
:101DB00010FC2B68029A1C121340364A9B009B5859
:101DC0000435FEF737FCA300FE1A3100200004930F
:101DD00002F0B4FA049B3060FE1A2F4B371D1B78BB
:101DE000002B02D0019EFEF7F4FB2B68029A1C1216
:101DF0001340284A9B009B580435FEF71BFCA300A8
:101E0000FF1A3900200000F0D5FD234B1B78002B72
:101E100002D0019EFEF7DDFB2B68029A1C121340D4
:101E20001C4A9B009B580435FEF704FCA300FF1AD4
:101E30003900200000F04AFD174B1B78002B02D020
:101E4000019EFEF7C6FB2B68029A1C121340114A32
:101E50009B009B580435FEF7EDFBA300FE1A3100F2
:101E60002000049300F01EFE049B3060FE1A0A4B13
:101E7000371D1B78002B02D0019EFEF7AAFB2B68B2
:101E8000029A1C121340034A9B009B580435FEF72C
:101E9000D1FBC04690980000BC020020A300FF1AAE
:101EA0003900200000F0F6FB224B1B78002B02D0FB
:101EB000019EFEF78EFB2B68029A1C1213401E4AED
:101EC0009B009B580435FEF7B5FBA300FF1A3900B1
:101ED000200001F0DFFB174B1B78002B02D0019E86
:101EE000FEF777FB2B68029A1C121340124A9B00E4
:101EF0009B580435FEF79EFBA300FE1A310020001C
:101F0000049301F0C7FB049B3060FE1A094B371D98
:101F10001B78002B02D0019EFEF75BFB2B68029A18
:101F20001C121340044A9B009B580435FEF782FBA9
:101F300009B0F0BDBC020020909800000023F7B566
:101F40005A1E0192002B07DA00F0E0FD01F016FEA8
:101F500001F0C4FE6423019300263000194B196878
:101F60008E4201DB019BEBE7174B1A68013291426D
:101F700000DC0022F0241A601D68144F6C43E35DFE
:101F8000002B1DD0E419022B16D0012B0ED10028F6
:101F900001D100F039F8F0226A430C4B0C499B1830
:101FA0005B68C31A8B4201D80223BB54F0235D4304
:101FB000064BEB5C022B03D12000FEF7E3FAD1E7DE
:101FC0000136CBE7C002002000000020D011002025
:101FD0009F86010000207047002070470020704756
:101FE0000020704701220020054B06491A61585015
:101FF0000330043158508018083158501A60704727
:1020000000800040040500000122034B1A64A8224E
:10201000D20098587047C0460080004010B5FFF7C6
:10202000F3FFFA21890004F0A5FA10BD10B50100F4
:10203000014803F00FFE10BD581100200048704702
:10204000989A000070B5054E0400335C0D008B4279
:1020500002D004F009FA355570BDC0460C060020C8
:1020600070B50024064D635D012B05D100212000D1
:1020700004F0FAF90023635501341A2CF2D170BD33
:102080000C0600200D20704735207047036870B59E
:102090005B100120052B12D8094A9B009C58094D62
:1020A0002B5D002B05D00021200004F0DDF900237A
:1020B0002B55200004F082F801234000184370BD26
:1020C000C49A00000C06002070B5036845685C10D7
:1020D0006D1004D40B4B9D4202DD1D0000E0002575
:1020E000192C0DD8084E335D012B05D0012120009D
:1020F00004F0BAF9012333552900200004F0ECF86C
:1021000070BDC046FF0300000C0600200B6870B5D0
:102110005D10192D16D80024012804DD4C68043CFC
:10212000624262415400094E735D9C4204D021001A
:10213000280004F099F97455280004F0C9F9042323
:10214000012800D00023180070BDC0460C060020F6
:1021500070B504000D0019280ED8084E335C012B11
:1021600004D0012104F080F9012333552900200017
:102170004D1EA94104F096F970BDC0460C06002022
:10218000436810B5191F4A424A41006811004010C7
:10219000FFF7DEFF10BD000037B56A46064B694603
:1021A00030CB30C203680220042B02D100F03EFB8A
:1021B00001E000F063FB37BD909A000010B5084CB9
:1021C000237D002B05D00021142004F04DF90023BD
:1021D0002375142004F07CF943425841800010BD5F
:1021E0000C06002010B5084CA37D002B05D0002163
:1021F000162004F039F90023A375162004F068F9BD
:1022000043425841800010BD0C06002070477047C3
:1022100010B5034A0421034801F028FA10BDC04656
:10222000080000205FA10000E12110B54902094823
:1022300003F0EEFDFFF7D6FE0A2003F0B9FF0023FE
:10224000FF21054A995401331A2BFBD100F0B2FD4E
:1022500010BDC046581100200C060020F8B50B4EEA
:10226000070030000D0003F013FE041EAC4200DD39
:102270002C003D00EB1B9C4205DD300003F012FEFC
:1022800028700135F6E72000F8BDC046581100203F
:1022900010B50100014803F0C3FD10BD5811002026
:1022A00010B5054C200003F0C9FDE12120004902D2
:1022B00003F0AEFD10BDC04658110020064B0120B2
:1022C0001A68064B06491A60C82200235200C850FB
:1022D00004339342FBD170473006002028060020CB
:1022E0002823002000B59BB00200054901A806F094
:1022F000FFFB01A801F082FB01F0F0FCFCE7C04607
:10230000DC9A000037B5184D04002868002801D079
:1023100005F0E2FFA400200005F0D4FF28600028AB
:1023200001D1124809E001AB984208D2104B0219C2
:102330006B440193934202D20E48FFF7D3FF042867
:1023400002D808302860083C2B680B4A1C1913601F
:102350000A4BC8221C600120002309495200C850C2
:1023600004339342FBD137BD30060020ED9A0000C4
:102370001CFCFFFF1D9B0000280600202C060020EF
:102380002823002070B50D4D0D4E2B684C1CA40069
:1023900036681C19B44203D90A20FEF7D5F80BE0C1
:1023A0002C601D00AC4201D904C5FBE70F220901D6
:1023B000104008431860180070BDC0462806002071
:1023C0002C0600200322CB1C70B50C00D91711403D
:1023D000C9180500891000220420FFF7D3FF00234D
:1023E000A34204DAE95CC21811710133F8E7E14352
:1023F0000023C917214041180B7170BD10B5830728
:1024000006D1042804D90F2304C81340042B03D099
:102410000E20FEF799F8014810BDC046B6A0000096
:1024200010B503240868044006D1042804D90F23FA
:1024300002681340042B01D00E2011E0FFF7DEFFED
:102440000378233B5942594110224018210006F0DD
:102450002FFC80239B05C218054B9A4203D91420F8
:10246000FEF772F802E001234000184310BDC04699
:10247000FFFFFF3F70B501240B680D001C4001D029
:102480005C1002E00D20FEF75FF8200004F074FB02
:10249000264904F05DFA05F037FE02F049FA002201
:1024A000234B04F0EBFF0023002204F01BFA01246D
:1024B0002B681C40002819D0002C01D05C1002E0D1
:1024C0000D20FEF741F8200004F056FB174904F0F8
:1024D0003FFA05F019FE02F02BFA0022144B04F02B
:1024E000CDFF0022134B04F08FFB18E0002C01D02D
:1024F0005C1002E00D20FEF727F8200004F03CFB02
:102500000A4904F025FA05F0FFFD02F011FA002255
:10251000074B04F0B3FF0022064B05F029FA05F043
:102520007BFD01234000184370BDC046D3023739FC
:102530000000D0400000E03F10B5034A02210348EC
:1025400001F094F810BDC04628000020889B0000D0
:102550000020704710B51E20FDF7F6FF10BD10B526
:102560001E20FDF7F1FF10BD10B51E20FDF7ECFF9A
:10257000002010BD10B51E20FDF7E6FF002010BDA5
:1025800010B51E20FDF7E0FF10BD10B51E20FDF7B1
:10259000DBFF10BD10B51E20FDF7D6FF10BD10B536
:1025A0001E20FDF7D1FF10BD7047000010B5034A93
:1025B0000921034801F05AF810BDC0463800002038
:1025C0009A9B00000123034A1360034A1068984055
:1025D000184370473C060020440600201E2800D9FE
:1025E0001A20084B8000C25801239340064A07492D
:1025F0001360074A1160074A07491160074A1360D0
:102600007047C046ECA300003806002008050050C3
:10261000540600204C0600200C0500501805005000
:10262000F0B5EFF310810123194083F31088134EA6
:10263000134AB4461268013A9340124A1468124A87
:102640001568124A002B15D0166803420BD026607D
:10265000C046C046C046C046C046C046C046C0464A
:1026600016682E6004E067463E601668084F3E60BC
:102670005B08E7E781F31088F0BDC046080500500D
:10268000C8000020540600204C0600203806002018
:102690000C0500500B6810B50200D80701D5581082
:1026A00001E0012040421823012A03DD4A68042A80
:1026B00000D10833024A1360FFF790FF002010BDDD
:1026C000C800002030B585B001AD0C2206492800B5
:1026D00005F00CFE0024285D01210134FFF7B2FC57
:1026E0000C2CF8D105B030BD269C0000F0B53B4C59
:1026F00085B0210003220C31684605F0F7FD21006A
:1027000009220F3101A805F0F1FDFFF787FC344BDA
:10271000344CC0182368984201D2002323602568F6
:10272000002D3ED12E006B4604339F5D0121380001
:10273000FFF788FC01360121380003F0B3FE092EB3
:10274000F1D100266B469F5D01213800FFF77AFC2E
:1027500001360021380003F0A5FE032EF2D1C82077
:1027600080000138C046C046C046C046C046C0468C
:10277000C046C046C046C046C046C046F1D1002152
:102780000520FFF75FFC00266B460021985D0136AF
:10279000FFF758FC032EF7D1FFF740FC1330206001
:1027A00019E0FFF73BFC23680025984213D305206E
:1027B00003F004FD0C4B0D4EC01801D4306000E056
:1027C00035603068032103F05FFF00230125084ACC
:1027D000306023601360280005B0F0BD269C000027
:1027E0001027000034060020C8FEFFFF440600202A
:1027F0003C06002010B50124044001D0441002E042
:102800000D20FDF7A1FE200010BD00000022054BA9
:1028100010B51A60044B1B68934201D001F026FEEC
:10282000002010BD480600207C10002070B508680C
:102830000D00FFF7DFFF04006868FFF7DBFF631E92
:102840000100042B14D8451E042D11D805226A431B
:10285000D318012215009D402B00064805682B4324
:102860000360054B1B68002B02D0200001F0FFFD28
:10287000002070BD480600207C10002070B508685C
:102880000D00FFF7B7FF04006868FFF7B3FF631E92
:102890000100042B14D8451E042D11D805226A43CB
:1028A000D31801229A401300064802689A43064B47
:1028B00002601B68002B03D00022200001F0D7FD2E
:1028C000002070BD480600207C100020F0B50500F7
:1028D00085B008680C00FFF78DFF0390022D08DD1E
:1028E0006068FFF787FF0700A068FFF783FF040019
:1028F00001E00124270005236343053B02930123E4
:1029000026000193231D9E4234DC3D003B1D9D4269
:102910002BDC731E042B23D86B1E042B20D8029BA8
:10292000039A591E019B49191A40204B0AD00122D3
:102930008A4019680A431A601D4B01221B68002B4C
:102940000ED009E001208840010018688843186013
:10295000174B1B68002B03D03100280001F087FDC6
:10296000019B01355B000193D0E7029B01360533E3
:102970000293C7E73D1D042D15D8012C13D1260065
:102980003300AB40094A11689943094B11601B6839
:10299000002B04D0781D0022210001F068FD0134D5
:1029A0000535062CECD1002005B0F0BD480600200E
:1029B0007C1000202D4BF7B51B680C00002B03D1B9
:1029C00001204042FFF70AFE01262468344219D054
:1029D000FF226310180212041040FF22611212023B
:1029E0000A40DBB210431843214B1B68202B06D151
:1029F000B440204BA40EA400E35800021843FFF794
:102A00000FFE30E0032525402DD1042C2BD90F23B8
:102A100022681340062B26D1FF27130901933F0498
:102A2000019B9D421FDAAB00E3185A68324218D06E
:102A3000531018023840FF21844609025012084002
:102A40006146DBB208431843094B1B68202B06D1B3
:102A50005200920E074B9200D35800021843FFF722
:102A6000DFFD0135DCE70020FEBDC0463806002052
:102A7000C8000020B49C0000086810B5C30703D547
:102A8000FFF7B8FE054B1860054B1B68002B03D001
:102A9000024B186801F0ECFC002010BD4806002035
:102AA0007C1000200868F8B5C30702D5FFF7A2FE26
:102AB0000BE0830726D1042824D90F2203681A408B
:102AC000042A1FD11B091DD000790300203B5E2B77
:102AD00018D80522002053430B4E9D18043AAB42F0
:102AE0000CD0052110249F5D3C4200D08018013994
:102AF000520064100029F7D10133F0E701234000B0
:102B0000184300E00120F8BDB49D00007FB5A44E3D
:102B10003368002B0BD1A34A1268002A07D1A24BBD
:102B20001B68002B00D139E1FFF7E0FD36E19F4D36
:102B30002A68002A2AD19C4A1268002A07D0FFF787
:102B4000D5FD002800D129E1FFF7BCFD05E0954A3D
:102B50001268002A01D1002BF6D1924B19681A0095
:102B6000002911D03468002C0ED101AD0C229049FF
:102B700028001C6005F0BAFB285D00210134FFF736
:102B800061FA0C2CF8D109E13368136000210D20A3
:102B900003F088FC00210E2003F084FC00210F20AC
:102BA00003F080FC2E68012E56D0022E00D19CE04E
:102BB000002E00D0ECE0013631007A4C042023686E
:102BC000994303F06FFC0421236805200B40594210
:102BD000594103F067FC1021236806200B4059423D
:102BE000594103F05FFC8021236809010B405942E1
:102BF00059410C2003F056FC8021236809020B4048
:102C0000594259410B2003F04DFC802123684902B1
:102C10000B40594259410A2003F044FC80212368AB
:102C200089020B4059425941092003F03BFC8021A5
:102C30002368C9020B4059425941082003F032FC75
:102C4000802321681B030B4059425941072003F0A0
:102C500029FC31000D2099E00221524C0720236805
:102C60000B405942594103F01DFC082021680140E6
:102C70000B005942594103F015FC80212368C9001B
:102C80000B4059425941052003F00CFC8021236878
:102C900049010B4059425941062003F003FC8021B1
:102CA0002368C9010B4059425941042003F0FAFB43
:102CB0008021236889030B40594259410A2003F0BF
:102CC000F1FB802321681B040B4059425941092024
:102CD00003F0E8FB31000C2003F0E4FB31000B2093
:102CE00003F0E0FB31000E2050E020212D4C0720A6
:102CF00023680B405942594103F0D4FB402123681B
:102D000008200B405942594103F0CCFB8021236835
:102D100009200B405942594103F0C4FB802123682C
:102D200049000B40594259410A2003F0BBFB802166
:102D3000236889000B40594259410B2003F0B2FB34
:102D40008021236889010B40594259410C2003F02E
:102D5000A9FB8021236849030B40594259410620B1
:102D600003F0A0FB80212368C9030B40594259415D
:102D7000042003F097FB802321685B040B40594239
:102D80005941052003F08EFB01210F2003F08AFB3F
:102D90002B680321581C03F05DFD29607FBDC046F0
:102DA00048060020400600203C0600205006002077
:102DB000269C0000012010B54042FFF70FFC0020C8
:102DC000FFF72EFC10BD000010B5034A092103488F
:102DD00000F04CFC10BDC046800000203E9C00006E
:102DE00030B502248025094B094AED009C505C59FE
:102DF000002CFCD0A124E400884204D28025ED0000
:102E000018514019F8E70021995030BD00E0014009
:102E10000405000010B5002804D19820A621400226
:102E2000890203E0A62080218002C902FFF7D8FFB3
:102E300010BD002802D0A6239B0201E098235B026C
:102E40001B6800201A0E532A01D11B02180A704772
:102E500030B501248025064A064BED00D450545964
:102E6000002CFCD001600021014AD15030BDC04689
:102E700000E001400405000010B5002802D0A620A3
:102E8000800201E098204002A6230902DB05090A1E
:102E90001943FFF7DDFF10BDF0B5012480250300C5
:102EA0000F4F08000F49ED007C507C59002CFCD0DE
:102EB0009C46002810DD5478167893782402344319
:102EC0001B0423431C00D37801381B0623436446AC
:102ED00008C40432A446ECE700237B50F0BDC04692
:102EE00000E001400405000070B505004B680A00D1
:102EF0009C1C2100FFF7D0FFA000281870BD000027
:102F0000154B1B68002B04D08021A623C9029B020D
:102F100003E0A621982389025B02002807D1191D2E
:102F20005B6802001B0E522B14D10A0012E0002233
:102F300081420FD903681B0E522B0BD14368023319
:102F40009B00C318994205D91A68110E0022522914
:102F500000D11A00100070475808002070B50020FA
:102F6000FFF7CEFFFF260500002808D003681C14D9
:102F70003440FFF7C5FFDA2CF6D10500F4E728004E
:102F800070BD00008022F0B55200A1B0002165485C
:102F900005F0B5F9802200215200634805F0AFF931
:102FA000624C23681A00039353425A411000049262
:102FB000FFF730FF039B0594002B01D15C4C00E030
:102FC0005C4C0020FFF7CAFFFF270500002D7CD0D6
:102FD0002A68131412123A403B4002921A000A3A2D
:102FE000092A42D84F4B029A995C002968D11022D5
:102FF000514805F084F92E00336802991A123A40BC
:10300000914217D11A143A400B2A06D0132A0CD039
:103010000A2A0FD1484B1E600CE03B40022B09DC12
:10302000454A9B00D3185E6004E01022002142480C
:1030300005F065F93000FFF763FF061EDCD13E4B5B
:10304000196800290FD02000FFF74EFF04003B4E07
:103050003168002903D02000FFF746FF0400384BF9
:103060000436B342F4D12F4B27E01A00153A082A50
:1030700026D82D4A0299565C002E21D1152B00D15D
:103080002E00280003681A143A40152A03D01D2A7E
:1030900007D1002605E0029A1B123B409A4200D15C
:1030A0000600FFF72DFF0028ECD1002E04D02000F1
:1030B0003100FFF719FF04001B4B0121029A9954BC
:1030C0002800FFF71DFF050080E70398FFF7B1FE1A
:1030D000411C0498FFF7D0FE059B1A4D049A2C6002
:1030E0001A60FFF7DDF8059B2C681B68002B02D0E7
:1030F000A6239B0201E098235B026420B421E41A1A
:103100006043490203F0C0FAB42252020300009265
:103110000D49220007A805F0EBFC07A800F06EFCA3
:1031200021B0F0BD580700205806002058080020A4
:103130000498020004300100B8240020BC240020C0
:10314000C82400205C0800209C9F0000F0B50020EF
:10315000B7B00024FFF7D4FE270005002600002D9D
:1031600020D0FF226B6828689C460233FF180312A8
:103170000136134011009C4200DA1C0002140A4080
:1031800003926246014001920091039A1C4904A8EF
:1031900005F0AEFC04A800F031FC2800FFF7B0FEFB
:1031A0000500DCE7174D2868FFF743FE3B00019060
:1031B00000943200144904A805F09AFC04A800F019
:1031C0001DFC124B1C682B68002B02D0A6239B020F
:1031D00001E098235B026420B421E41A60434902B1
:1031E00003F052FAB422520203000092084922006E
:1031F00004A805F07DFC04A800F000FC37B0F0BD89
:10320000D29F000058080020E69F00005C080020C4
:10321000B79F000070B50020FFF70BFE04000120EF
:10322000FFF707FE844200DA04000A4B1E6875426D
:10323000754128001D60FFF7EDFD002E01D0064B03
:1032400000E0064B064A2800611C1360FFF714FEDD
:1032500070BDC046580800200430010004980200E8
:103260005C080020F8B50020FFF7E3FD070001200F
:10327000FFF7DFFD3E00224D0643224C0CD180219A
:103280009820C9024002FFF7ABFD01213000FFF793
:10329000F3FD2E601C4B2FE0874208DD0023A621A2
:1032A0002B60194B890223602368002011E0012361
:1032B00080212B60154BC9022360F5E71A68551C65
:1032C00018D0120E522A07D101205A6802329200F9
:1032D0009B188B42F2D311E0002800D023600C4CE5
:1032E0000C49200005F030FC2000FEF79FFEFFF7A0
:1032F00091FF04E0002802D0236000E02160F8BDC7
:10330000580800205C0800200430010004980200E6
:10331000042500201BA00000F0B585B00392032215
:103320000333DC1714402A4EE3189C1033680190D5
:103330000291002B02D08022D20201E0A62292024A
:10334000244FA51C3B68AD005B199A4217D2FFF7CA
:1033500019FE3368002B02D08022D20201E0A6229F
:1033600092023B685B199A4209D21B4C1B49200010
:1033700005F0EAFB2000FEF759FE002026E0029B44
:103380003E681B06190C6B461A7BA423DB0513430E
:10339000019A0B431104FF2212041140194330001B
:1033A000FFF756FD3300301D0833210001933B60C9
:1033B000FFF74EFD002C04D00A9A21000198FFF778
:1033C0006BFD3000019B083D5D193D6005B0F0BD0F
:1033D000580800205C0800200425002044A00000BC
:1033E00010B5FFF7CFFD10BD70B59AB0FFF73AFFEB
:1033F000FF22264CD2000021200004F080FF002094
:10340000FEF7DCFE042804D10020FEF7EBFE0428C2
:1034100031D00020FFF7A2FDFF25002600281AD09A
:1034200003681A142A400A2A08D11A122A40FF2ACD
:103430000ED0D200A1180B71A05009E0132A07D1B9
:103440001B122B40FF2B03D0DB00E2181671E65055
:10345000FFF756FDE2E7FF210200C90023580830BC
:103460005D1EAB41D2188842F8D1094901A805F088
:103470003FFB01A802E0FFF7CDFE064800F0BEFAD0
:10348000054800F0BBFA1AB070BDC046301B0020E2
:103490006BA0000087A000007FA000000020704704
:1034A0000120704700487047E02400200048704722
:1034B00033F8FFFF10B50449044805F045FB242309
:1034C0000348036010BDC0464AA10000CC24002080
:1034D000C82400200020704700207047002070475B
:1034E0000020704700207047002070470020704780
:1034F000002070470020704710B5034A0E21034892
:1035000000F0B4F810BDC046CC0000204FA1000070
:10351000044A05491368C85401339B059B0D136089
:103520007047C046640C002060080020114A70B546
:103530001368114C984211DA015D451CFA390129D2
:1035400006D8AB4206DD2118497801391F2901D977
:103550002800EFE70100251A461C02D10023136062
:1035600006E0665C6E5401318B42FADC181A10607A
:1035700070BDC046680C0020700C002010B5FEF72E
:1035800043FD064B1A68904201D200221A601B6864
:10359000C01A034B83428041404210BD6C0C002096
:1035A000204E000010B5094C094A23681268934266
:1035B0000BD0084AD05CFEF76BFE002805D02368CC
:1035C00001339B059B0D2360EDE710BD70100020BB
:1035D000640C00206008002010B50400064B074A68
:1035E0001B6812689B1ADB439B059B0DA34202DA02
:1035F000FFF7D8FFF2E710BD640C00207010002028
:10360000F7B506000191151E2FD05768B800441C6D
:103610000630FFF7E1FFFB20FFF77AFF1C20FFF7E2
:1036200077FFF0B2FFF774FFE0B22412FFF770FFEC
:10363000E0B2FFF76DFF6B461879FFF769FF0026D0
:10364000BE4212DAB300EB189C680136E0B2FFF715
:103650005FFF2012C0B2FFF75BFF2014C0B2FFF77C
:1036600057FF200EFFF754FFEAE7F7BD70B5074D8F
:103670002C68092C08DC0C236343054E0134985157
:10368000F31859609A602C6070BDC0467410002019
:1036900068250020F0B589B004900E0001284BDDAC
:1036A000284B08680293830709D1042807D90F2300
:1036B00002681340042B02D1FEF7A0FE0290214BBA
:1036C00070680393830709D1042807D90F23026880
:1036D0001340042B02D1FEF791FE039000271A4BF2
:1036E0001A4D1B680593059B9F4225DA2B1F0299F3
:1036F000186805F01FFA00281BD12B686C68069328
:103700000190019B069A934213DA2068039907946B
:1037100005F010FA0834002807D131000498079BFF
:1037200008315B680238984709E0019B0133019337
:10373000E7E701370C35D6E71B20FCF705FF09B09A
:10374000F0BDC046B6A00000741000206C2500201B
:1037500010B5FFF739FBFEF75BFDFEF7EDFEFEF758
:1037600025FFFFF7C9FE00F0FFFC00F083FE10BD4F
:10377000962210B512010021034804F0C0FD00227A
:10378000024B1A6010BDC046D0110020C0020020BC
:10379000064B074A1B6812689B1ADB439B059B0D6F
:1037A0000122834200DC002210007047640C0020DC
:1037B00070100020F8B505000C0016001F1E0ED179
:1037C0000320FFF7E5FF002827D0FA20FFF7A0FE2F
:1037D000E8B2FFF79DFEE0B2FFF79AFE1DE0501D34
:1037E000FFF7D6FF002818D0FB20FFF791FEE8B2C4
:1037F000FFF78EFEE0B2FFF78BFEF0B2FFF788FE18
:103800003012C0B2FFF784FE3C00E31B9E4204DD91
:103810002078FFF77DFE0134F7E7F8BD70B500248E
:10382000F0250B4B1B689C420EDA2A006243094BC1
:10383000D3181A78002A05D05978002311201A00CD
:10384000FFF7B8FF0134ECE7FFF792FF70BDC04609
:10385000C0020020D01100200123F3B50400FFB006
:103860000D0010001A420DD002AA1370431002A9D5
:10387000537042121B0E40148A700B71C8700B00FB
:10388000052273E0032313401ED1042A1CD90F2202
:1038900001680A40042A17D1023302AA1370FEF706
:1038A000ADFD060005F058F9F823FF33984200DD1E
:1038B00018000023834205DA01335A1EB25C02A9C4
:1038C000CA54F7E7421C50E0042801D0002809D16F
:1038D000032302AA04381370434243415370130078
:1038E000022243E0002B45D1042843D90F2102686E
:1038F0001140052912D1043302A90B70F8231209D3
:10390000FF3392009A4200DD1A00002393422BDA23
:103910000133C118C97802AEF154F7E7062929D15D
:1039200001390E00120956430196F826019FFF3611
:10393000B7421FDC02AE31700136934213DA012721
:10394000013399004158394201D0394100E00A4918
:10395000012737700F127170B7700F14090EF770CE
:1039600031710536E9E7019A013202AB29002000E6
:10397000FFF720FF7FB0F3BD19FCFFFF70B5F02308
:10398000050000240D4A1800604380184178A942C0
:1039900003D001340A2CF6D10FE0F022002104F00C
:1039A000AEFC074A1368013BA34200D11460002318
:1039B00029001A001120FFF7FDFE70BDD011002074
:1039C000C002002010B5B2B002236A460400137092
:1039D00005F0C2F8C72800DDC7200023834205DABE
:1039E000694601335A1EA25CCA54F7E7421C6B4673
:1039F000FE211420FFF7DEFE32B010BD30B5B3B0AB
:103A000002236A460500137005F0A6F8041EC72CB1
:103A100000DDC7240023A34205DA694601335A1E9C
:103A2000AA5CCA54F7E720003230FFF7D5FD621CCC
:103A30006B46FF211420FFF7BDFE33B030BD000000
:103A4000F7B5234B06001B68F020009300232149A3
:103A5000009A93420ADA02005A438A185478B44210
:103A600002D11278002A31D10133F1E70024F0238A
:103A70001A00624301920199164A55182F78002FB7
:103A800006D001340A2CF3D11348FFF7B7FF1DE02D
:103A9000F0223900280004F032FC02230D4A01997B
:103AA000EB6053540D4AF1008A58009B6E70AE7063
:103AB000AA602F616F61A34202DC054B01341C60D8
:103AC000002331001A001020FFF774FEF7BDC04636
:103AD000C0020020D01100200AA20000301B0020EC
:103AE00010B5FFF79BFE0024064BE200D3181B79AC
:103AF000043B012B02D8E0B2FFF7A2FF0134FF2CF8
:103B0000F2D110BD301B0020F7B50E0000247F2538
:103B10000190194BE200D1180979062901D0032937
:103B200026D1985883682B401C2B21D1C3681A00DA
:103B30002A40042A1CD102692A40192A18D11B0ADA
:103B400001339B000C30C018FEF758FC070005F04D
:103B500003F80023B0420BD19E4206DD019AF95CC6
:103B6000D25C914204D10133F6E7E0B2FFF768FF7F
:103B70000134FF2CCDD1F7BD301B002070B5FEF70E
:103B800043FA184B1A68904201D200221A601A6850
:103B90001549821A8A4223D918600020FEF70EFBCD
:103BA000444244416042072404430020FEF71AFBCC
:103BB000002810D0082600250C4BEA00D3181B79EA
:103BC0009C4201D0B34202D1E8B2FFF739FF013580
:103BD000FF2DF1D104E0631C02D001267642EAE712
:103BE00070BDC046600C00200F270000301B002075
:103BF00037B500240500FFF711FE01A80194FEF778
:103C0000CBFA21002000FEF701FEFEF77FFFFEF752
:103C1000FDFAFEF7FCFAFFF7CDF8FEF721FAA54210
:103C200004D0FEF74BFB0248FFF7E8FE37BDC04665
:103C30001FA20000002310B501001A001120FFF799
:103C4000B9FD10BD07B56B46197069465A7013125D
:103C50008B701314120ECB700A716B460100052293
:103C60001320FFF7A7FD07BD10B50A0001001220C1
:103C7000FFF7F2FD10BD70B5050008000C003230F2
:103C8000FFF7AAFC2B00220000211B20FFF792FD6A
:103C900070BD10B50C000300110014202200FFF7C6
:103CA00089FD10BD70B506000020FFF729F900243A
:103CB000FF25002810D003681A142A40152A05D1C0
:103CC0001B122B40B34204D1040002E01D2A00D194
:103CD0000024FFF715F9ECE7200070BDF0B5802750
:103CE0009DB0FFF75FFCB64DB64C2868FF00391A4F
:103CF0002018FEF7B3FA2B680600C3182B60002BC0
:103D000000D1D9E1002E0DDD2868391A2018FEF700
:103D1000A5FA2B6806001B182B60FEF775F9AA4B55
:103D20001860EFE72378FA2B00D00CE12B68022B08
:103D300006DCFFF723FC002800D1BDE10120B6E13D
:103D40006078A5780238182800D9FAE002F008FC5B
:103D50000D1E22262932F93D67F96F83D4E5F9F962
:103D6000F9F9F9F9F9F9F9F9F300FF2D00D1E8E0D3
:103D70002800FFF703FE00229449EB005A50CB18AD
:103D80001A7129000092130013204DE02800FFF75C
:103D900057FED6E02800FFF7F1FDD2E0FFF7A0FEC6
:103DA000CFE0FFF73BFD0020FFF722FF8848FFF739
:103DB00025FEC6E0632D00D9C3E0864BAA00D25889
:103DC00029001520FFF748FDBBE000242000FFF785
:103DD00069FF071E03D10134642CF7D1B1E008302C
:103DE00004F0BAFE06000530FFF7F6FBFB20FFF7F4
:103DF0008FFB1D20FFF78CFBE0B2FFF789FBF0B2D1
:103E0000FFF786FB3012C0B2FFF782FB0025AE42FF
:103E1000E1DD7B19187AFFF77BFB0135F7E700211D
:103E20001D200B000A000091FFF776FA89E0FEF7EB
:103E300005F903AC684A64210090684B200004F047
:103E400025FE02232000237004F086FE23000200DA
:103E50000021162073E000245C4AE300D558002DB1
:103E600046D06B689E00701DFFF7B6FB2B00002547
:103E70003200083321000120FFF79CFC0020FFF7EF
:103E80003FF82E002F0000281DD0FF2103681A12D2
:103E90000A40A24214D11A140A400B2A07D10B403F
:103EA0000DD0012B09D0022B00D103E108E0132A29
:103EB00006D100252E002F0002E0060000E00700DA
:103EC000FFF71EF8DFE7002E04D0320001212000AA
:103ED000FFF796FB002D04D02A0002212000FFF7F7
:103EE0008FFB002F04D03A0000212000FFF788FB51
:103EF0000134FF2CB0D124E00024FFF78FFC220016
:103F0000210000942300DA20FFF706FAFF222100A7
:103F1000D2002E4804F0F3F913E0012D02D1FFF78F
:103F200015F90EE0022D02D1FFF75AFA09E001203F
:103F3000FFF75EFE05E0002329001A001A20FFF7B4
:103F400039FC0320B3E0FB2B00D0F7E62A68042AF3
:103F500000DCEEE62679E078214B360206439E42ED
:103F600000DDEBE6331D9A4200DCE2E6E35CFE2B6B
:103F700000D0E3E66378A578711E1B2B5DD004D8D2
:103F8000012B08D0082B2DD090E01D2B64D058D3E6
:103F90001E2B7BD08AE0FF2D00D187E02800FFF7A1
:103FA000EDFC67790634B31E290000943A000A201C
:103FB000FFF7B2F9054BED00E8505D192F7175E080
:103FC000680C0020700C00206C0C0020301B0020BE
:103FD0002EA200002823002045A2000040A20000DD
:103FE000F6030000632D61D86079022813D00328FE
:103FF0001BD001285AD1A71D7A78A479BB78120268
:1040000022431B0413431A00FB78AD001B06134325
:104010005B0003430EE0002948DDB11EA01DFEF742
:10402000D1F9264BAD00E85040E0A379AD005A1E0F
:1040300093419B00214AAB5038E0601DFFF764FDBF
:1040400034E06279FF2D31D0022A2FD80634B31E16
:10405000009429000B2016E00B1E632B00DD632368
:10406000002203A8934204DDA1184979815401324A
:10407000F7E7D9430022C917194041180A70009088
:10408000290015200133FFF747F90FE0012D0DD16D
:1040900000290BDD6379002B03D0322B02DD3223A4
:1040A00000E02B0064225343054A1360701DFFF7A4
:1040B0003DFA01E0050003E71DB0F0BD2823002014
:1040C000040000200120704710B5064C200000F0CD
:1040D00007FB0549200000F027FB0122034B1A6073
:1040E00010BDC046A0100020801A060078100020E5
:1040F00010B501210D20FDF7A5FF01210E20FDF7D0
:10410000A1FF00210F20FDF79DFF044C200000F0CF
:1041100023FA1021200000F03BFA10BD8C10002083
:1041200010B504680D20E30703D56410FF2C03D9F4
:104130001720FCF709FA06E0FFF7DAFFE1B20248C0
:1041400000F048FA002010BD8C10002010B5FFF7D9
:10415000CFFF0021034800F03DFA0123400018433F
:1041600010BDC0468C10002010B5034A072103483B
:10417000FFF77CFA10BDC0463C0100204CA20000B5
:10418000F8B5012306681E4205D045681D4202D0DD
:1041900084681C4201D10D2004E076106D10802E41
:1041A00003D91520FCF7D0F91DE01620FF2DF9D812
:1041B00064101720FF2CF5D80B4B1B68002B01D186
:1041C000FFF782FF094FF1B2380000F035FBE9B28A
:1041D000380000F046FAE1B2380000F042FA380048
:1041E00000F094FB0020F8BD78100020A010002003
:1041F000F7B501242300A04237DD0A68144234D009
:104200001B4B55101B684C68002B01D1FFF75CFF5E
:104210000127184EE9B2300000F00EFB3C4205D0F9
:104220003C413000E1B200F01CFA1AE003252540C1
:1042300017D1042C15D90F2322681340062B10D157
:1042400013090193019B9D420BDAAB00E3185968F7
:10425000394204D04910C9B2300000F002FA0135E9
:10426000F0E7300000F052FB00231800FEBDC0460E
:1042700078100020A0100020144B70B51B680500BA
:104280000E00002B01D1FFF71FFF114CEDB22900EA
:10429000200000F0D1FAF1B2200000F0E2F9002194
:1042A000200000F0D5FA002801D040420CE00122A5
:1042B0002900200000F0BBFA200000F0C8F9002817
:1042C000FAD0200000F0C8F970BDC0467810002078
:1042D000A010002010B501240368234202D04168D9
:1042E000214201D10D2004E058104910802803D943
:1042F0001520FCF729F907E0FF2901D91620F8E776
:10430000FFF7BAFF4000204310BD10B50721182069
:10431000FFF7B2FF7F2801DD0138FF3803007F334C
:1043200001DA7F20404264237F215843494202F052
:10433000ABF9012340424000184310BD10B50821DD
:104340001820FFF799FFC30F1818012340101530EC
:104350004000184310BD10B505211820FFF78CFF51
:104360007F2801DD0138FF3803007F3301DA7F2029
:10437000404264237F215843494202F085F90123DA
:104380004000184310BD10B503211820FFF774FF3B
:104390007F2801DD0138FF3803007F3301DA7F20F9
:1043A000404264237F215843494202F06DF90123C2
:1043B0004000184310BD0000F8B501263400B0429B
:1043C00036DD0F683E4233D04D68AB0730D1042D47
:1043D0002ED90F232A681340062B29D1154B1B68B1
:1043E000002B01D1FFF770FE0024354204D12B6869
:1043F0001C09202C00D920240F4E7F10F9B2220076
:10440000300000F014FAA700EF19AF420DD03000D1
:1044100000F01DF90028FAD0300000F01DF901234A
:104420004000184368600435EFE70120640004434E
:104430002000F8BD78100020A01000200020704758
:104440000020704700207047002070470020704710
:104450000020704700207047002070470020704700
:104460000020704700207047002070477047704759
:104470007047000010B5034A0C210348FFF7F6F817
:1044800010BDC046740100208DA2000010B5FDF7DC
:10449000CBFE0648FDF736FFFFF75AF90448FFF751
:1044A000ADFAFEF7A1FFFFF71BFB10BD46050000AC
:1044B00003A3000010B5FDF741FD10BD70B5002548
:1044C00004AC24780573A94205D10A4B0A4A23217A
:1044D0000A4803F08BFE01600949920052589B0084
:1044E00002715B588371A3005B588560437102239E
:1044F000C37170BD58A300001BA3000066A3000099
:10450000ECA30000037B002B04D14373837303618E
:1045100001330373704700001FB50191A0210024EF
:104520000068C900D2B24450012A07D0A24203D089
:10453000032A05D1042202E0022200E006221343EE
:10454000034A8350034B019AC250012343501FBDBD
:10455000540500002405000010B50400FFF7D2FF49
:10456000A1222368A179D20099506179064A2000DE
:104570009950217904329950044B19685A689B6804
:10458000FFF7CAFF10BDC0460C05000080100020D8
:104590004BB2002B0CDB80233F290CD81F290CD8F1
:1045A0000F290CD807290CD803290CD81B060BE0BF
:1045B00080239B0408E0DB0406E01B0504E05B05A8
:1045C00002E09B0500E0DB050168014A8B50704763
:1045D000240500000368074A99501A00FC32D1688C
:1045E0000029FCD0A321C90058580023C0B2D360D1
:1045F0007047C0461C05000007B58022074BD20556
:104600001A6000229A6002321A7111230E3200934E
:10461000034905330348FFF751FF07BD8010002011
:10462000003000408C100020F8B505000E00170087
:104630000024BC4208D02B68315D1B6828009847D5
:10464000002801D00134F4E72000F8BD704710B510
:104650001C3001F02BFB10BD10B51C3001F018FB15
:1046600010BD70B5437E0D00002B05D064300400F2
:1046700001F02BFB002801D0002004E020002900DD
:1046800001F0F7FA012070BD10B51C3001F014FBE9
:1046900010BD0000F7B50193FA23002504009B002C
:1046A00083600D4B4560083303601C300F0016001B
:1046B00001F0D4FA2000643001F0D0FA074AB600C5
:1046C000B35827616375019B20009B009B5865765A
:1046D000A576A375FEBDC046CCA30000ECA30000E8
:1046E0000123A022C375837D0C49C133FF33D2055A
:1046F0009B009950437DC133FF339B009950CC21DF
:104700000369074A490499500521243A9950817D4B
:1047100008329950417D034A995070470C060000B9
:10472000240500000C050000A02302690020DB0026
:10473000D0500948814204D90848814204D9CD218A
:1047400003E0CC21490401E08021C9040448115050
:104750000521D1507047C046A086010090D00300CB
:1047600024050000F7B5050000200C0001938242EB
:104770005CD0161E402E00D940262F001C37380072
:1047800001F082FAB1222B69D20080219C500122D3
:1047900089005A50A97E002901D11A621A600024AA
:1047A000731E2A69A34206D1019B002B03D08023EC
:1047B00002219B00D150012313621300FC33D968FE
:1047C000002902D1996A0029F9D0996A00290AD1F1
:1047D000D960A323DB00D1583800C9B2013401F0FD
:1047E00048FAA642DCD8019A2B69002A04D11A00A3
:1047F000FC32916A00290AD001210022AA7659616F
:104800001900FC3188680028FCD08A6007E001218B
:10481000A976D961D16C0029FCD00021D164FC3388
:104820009A6A002A01D000229A62E0B2FEBD10B559
:104830000123FFF797FF10BD0300AC3310B5040050
:104840001970643001F020FA0123637610BD000076
:10485000F8B500220D0001004276AC310369040076
:104860000878B121C9005850802189005A5001327E
:104870001A629A6026006436300001F017FA0028A8
:104880000ED03000276901F003FA1E4BF85023695F
:10489000FC331A6A002A0CD19A6A002AF9D008E07F
:1048A0002369002D0AD11A00FC32916A002905D132
:1048B0000EE09A6A002AF3D11A62DBE701225A61FC
:1048C0001A00FC3291680029FCD00021916006E0BA
:1048D0000121D961D16C0029FCD00021D1641A00DA
:1048E0000020FC32916A81420BD0074990625A58ED
:1048F00002305A50824204D0043A534253410230AB
:10490000C01AF8BD1C050000C404000010B5012148
:10491000FFF79EFF10BD000010B5132312220249BD
:104920000248FFF7B7FE10BD00400040A010002075
:1049300030B5214A4B0087B05B0893421EDD1F4A09
:10494000934205DD02000B0003F012F807B030BD02
:1049500002AA00F035F803231840049A059B0128A9
:104960001ED0022811D000281FD00298039900F011
:104970002DFA80231B069C466144E7E700230022B2
:104980000093002300F088FFE0E7012402980399D8
:10499000009400F081FF80231B069C466144D5E70C
:1049A0000298039900F012FAD0E7012402980399C3
:1049B000009400F071FFC9E7FB21E93FFFFFEF7FA3
:1049C000F0B54E4657464546E0B4DC4B4E0090B03D
:1049D0001700894676089E4200DC81E0D84B9E4253
:1049E00020DCD84A002900DC89E1D74B02F0C0FF67
:1049F000D54B04000D009E4200D18AE0D34AD44B2F
:104A000002F0B6FF02000B0020003A607B60290034
:104A100002F0AEFFCD4ACE4B02F0AAFFB860F960BB
:104A2000012066E0CB4B9E4200DC8DE0CA4B9E42EB
:104A300065DCCA4932158A46924453461B05F51A6D
:104A40002900040003F0E8FA03F01CFB02000B004D
:104A5000200029000A920B9302F08AFF0022C04B2B
:104A600002F00CFD0290039103F0D6FA03F00AFB6A
:104A700004000D0002000B00029803990C940D95A0
:104A800002F076FF0022B64B02F0F8FC0022002371
:104A90000E900F9101F002FF002800D14CE100239D
:104AA00000222000290001F0F9FE0222431E984155
:104AB000131AAC4A3900019202220AA80092524607
:104AC00000F09EFA4B46002B13DA80221206944621
:104AD0007B68404263447B60FB686344FB6008E0A2
:104AE00002000B003A607B60002200230020BA60C5
:104AF000FB6010B01CBC90469946A246F0BD020077
:104B00000B0002F035FFB860F96038607960002072
:104B1000EFE7D3228E4B520502F02AFF924A934BC5
:104B200004000D0002F024FF02000B0020003A6098
:104B30007B60290002F01CFF8B4A8C4B02F018FFAF
:104B4000B860F9600120D4E700F056FF884A894B2D
:104B500004000D0002F092FC0022874B02F054F892
:104B600003F05AFA804603F08DFA764A764B0690A7
:104B7000079102F083FC02000B002000290002F0E4
:104B8000F7FE734B02900391069807996F4A02F063
:104B900075FC434604000D00049405951F2B30DC82
:104BA000013B764A9B009B589E422AD002000B0094
:104BB0000298039902F0DCFE02000B0005000C00D5
:104BC0003A607B60029803992A00230002F0D0FE2D
:104BD000049A059B02F0CCFE06000B003200BA607E
:104BE000FB604B464046002B00DB82E780231B0620
:104BF0009C46644461443D607C60BE60F960404214
:104C000077E7049A059B0298039902F0B1FE0B0026
:104C100002003A607B604B0036155B0D05000C000E
:104C2000F31A102BCEDD06980799D322484B520574
:104C300002F024FC04000D0002000B00029803990E
:104C400002F096FE02000B00029803990892099365
:104C500002F08EFE22002B0002F08AFE04000D00FE
:104C600006980799404A414B02F008FC22002B00AD
:104C700002F07EFE02000B0004900591089809994D
:104C800002F076FE02000B003A607B604B005B0D89
:104C9000F61A0500089A099B0C0002920393312E24
:104CA00090DD06980799B822304B920502F0E6FB9A
:104CB00004000D0002000B000298039902F058FE58
:104CC0000A0001001300029103920200089809995A
:104CD00002F04EFE22002B0002F04AFE04000D00FE
:104CE00006980799264A274B02F0C8FB22002B00A2
:104CF00002F03EFE02000B000492059358E7124BAF
:104D000001F082FF104B04000D009E423CD00F4A80
:104D10000F4B01F079FF02000B0020003A607B602E
:104D2000290002F025FE094A094B01F06DFFB86029
:104D3000F96001204042DCE60323BAE6FB21E93FAB
:104D40007BD9024000004054FB21F93F3163621AD5
:104D500061B4D03DFB213941FFFFEF7FEAFBFFFF4C
:104D600000007041E8A400007370032E8A19A33B71
:104D700083C8C96D305FE43F0000E03F68A40000D5
:104D8000C14920259A837B39D3220D4B520501F06E
:104D90003BFF0C4A0C4B04000D0001F035FF0200F4
:104DA0000B0020003A607B60290002F0E1FD054A1B
:104DB000054B01F029FFB860F9600120404298E6F8
:104DC00061B4D03D7370032E8A19A33BF0B54F46F2
:104DD0004646C0B487B000920193754B4F008146A0
:104DE00088467F089F4263DC03F016F9002800D153
:104DF000DAE04A4643464846414602F03FFB04009B
:104E00000D006C4A6C4B02F039FB6C4A6C4B01F0A4
:104E1000FBFE22002B0002F031FB6A4A6A4B02F0D3
:104E2000A7FD22002B0002F029FB684A684B01F025
:104E3000EBFE22002B0002F021FB664A664B02F0DB
:104E400097FD22002B0002F019FB644A644B01F02D
:104E5000DBFE22002B0002F011FB029003910022E6
:104E6000604B2000290002F009FB029A039B060018
:104E70000F002000290002F001FB009A019B0400B2
:104E80000D004846414602F0F9FA02000B002000EE
:104E9000290002F06DFD02000B003000390002F025
:104EA00067FD02000B0000204F4902F061FD70E039
:104EB00002000B0002F0E2FA04000D003D4A3E4BF6
:104EC00002F0DCFA3D4A3E4B01F09EFE22002B0030
:104ED00002F0D4FA3B4A3C4B02F04AFD22002B0080
:104EE00002F0CCFA394A3A4B01F08EFE22002B0038
:104EF00002F0C4FA374A384B02F03AFD22002B0088
:104F000002F0BCFA354A364B01F07EFE2B0022003F
:104F100002F0B4FA354B029003919F429FDD344B6F
:104F200000229F423ADC334900207B182E491600AC
:104F30001F0002F01DFD049005910022294B200066
:104F4000290002F09BFA32003B0002F011FD029AA8
:104F5000039B06000F002000290002F08FFA009A40
:104F6000019B04000D004846414602F087FA02000A
:104F70000B002000290002F0FBFC02000B003000B7
:104F8000390002F0F5FC02000B000498059902F0CC
:104F9000EFFC07B00CBC90469946F0BD164B0026BE
:104FA00004920593154FC8E700200F49F1E7C0466A
:104FB000FFFF3F3ED43888BEE9FAA8BDC4B1B4BDF6
:104FC0009EEE213EAD529C804F7E923E9015CB19B5
:104FD000A001FA3E7751C1166CC1563F4C5555554C
:104FE0005555A53F0000E03F0000F03F3233D33F6E
:104FF0000000E93F0000E0FF0000E73F0000D23F73
:10500000F0B556464D4644465F46F0B48E4CA54436
:10501000099119001400A89A0B938C4B9200D25856
:105020000B000290013BE01E18211D0016000892A3
:10503000009301F029FBC3430200DB171A40130061
:10504000110001330E929A009B1ADB001B19069384
:105050004C1B761918D4A99BA5009C46361926AF7F
:105060006544013607E0286803F00CF8013403C7F3
:105070000435B44208D0002CF5DA002000210134B8
:1050800003C70435B442F6D1089B002B01DA00F0C7
:10509000F9FB76AB19008B4626AA9146089A0A932B
:1050A0000132D2009344029A9A469046009BDB005C
:1050B000994408339844009B002B00DAB5E14C4634
:1050C00000260027029D2268636803CD02F0D6F90E
:1050D00002000B003000390001F096FD083C06008C
:1050E0000F004545EFD15346C0C39A4608239C465E
:1050F000E144DA45DFD10899554A0B0094466344F0
:105100009B0012A884461A000298624483460D92BE
:105110000B9A0433D200634493440F930591059A8C
:105120000A98D30019000C938C46030063441E6850
:105130005F68002A34DD12AB99461300454A804669
:1051400094466344DB00984474AB9A460022424B79
:105150003000390002F092F902F05EFF02F092FF97
:1051600000223E4B04000D0002F088F902000B0003
:105170003000390002F0FCFB02F04EFF4B4601C349
:105180009946434620001A685B68290001F03CFDFF
:1051900008235B429C46E04406000F00D045D5D171
:1051A000069B30001A003900994600F0C1FCFF232D
:1051B00000229B0504000D0002F060F900F020FCC5
:1051C0000022274B02F05AF902000B0020002900B0
:1051D00002F0CEFB04000D0002F01EFF804602F03C
:1051E00051FF02000B002000290002F0C1FB4C46D9
:1051F00006000F00002C00DCF8E0059B18205A1E6A
:10520000920012AB9B58001B190001418844814059
:105210005B1A12A98B501722121B13410793079B8D
:10522000002B4BDD01239C46059BE044002B00DC5A
:10523000F2E280251096119712AB00210024094854
:105240006D04059F19E0C04684FDFFFFF0A5000036
:10525000FEFFFF3FFFFFFF1F0000703E0000704198
:1052600000002040FFFFFF00002A02D0AA1A1A60A7
:105270000134013104338F4209DD1A68002CF3D068
:10528000821A01311A60012404338F42F5DC109E2A
:10529000119F069B002B0EDD012B00D1B1E0022BEC
:1052A00009D1059B12A95A1E920012AB9B5810936C
:1052B0009B029B0A8B50079B022B7ED0002300226F
:1052C0003000390001F0EAFA059B002800D16BE2BA
:1052D00008995A1E914210DCBF490F988C4612A9BA
:1052E00063448C4600219B0063441C68043B2143BB
:1052F0008342FAD1002900D0B5E0089B12AA013BF5
:105300009B00D358002B00D084E201220D9B043B6C
:10531000596801320029FAD005990B008C460133F7
:1053200062440792934242DC0E9A9446A99A6344DF
:1053300092460B9A9B00944626AA90469A44059B57
:105340000A9A6344DB0098440C9B94469946079B59
:10535000E144DB00634405935346186802F092FE73
:10536000434618605960009B002B23DB444600260F
:105370000027029D2268636803CD02F07FF80200D7
:105380000B003000390001F03FFC083C06000F0024
:105390005D45EFD14B469E60DF6004239C4604339D
:1053A000E2449C46059BE144E0449945D4D1079BE7
:1053B0000593B4E600260027ECE732003B0000200E
:1053C000864902F0D5FA06000F00002C00D175E7DF
:1053D000069A0020814900F0ABFB02000B00300070
:1053E000390002F0C5FA06000F0067E7069B002BA4
:1053F00012D1059B12AA013B9B00D558EB150793D0
:105400000DE7059B12A95A1E920012AB9B581093F0
:105410005B025B0A8B504EE70022714B01F062FA8F
:1054200000280ED10023079348E7534600260027A3
:10543000C0C39A4608239C46E144DA4500D03AE6C8
:1054400059E601239C4601330793059BE044002B5A
:1054500000DDEEE632003B000020604902F088FAF1
:1054600006000F002AE743460B93069B12A8183B41
:10547000190006939300C3580092002B0FD1564891
:105480001300844612A8634484469B006344043B93
:105490005868013A18390028F9D000920691069A06
:1054A00000204E4900F044FB009B04000D00002B3F
:1054B00000DAB3E112AA94469F00DB0067449C46E1
:1054C0000A9A0593624493461600386802F0DAFDA2
:1054D00022002B0001F0D2FF424B306071600022AD
:1054E0002000290001F0CAFF083E74AB04000D0043
:1054F000043FB342E9D100239A464EAB0293089B86
:1055000099464B4600260027002B21DB8020364B96
:105510005D469846C005354900260027002408E06E
:1055200008239C460835E044A24511DB4346186831
:1055300059682A686B6801F0A1FF02000B00300077
:10554000390001F061FB013406000F00A145E7DAE4
:10555000029A53469446DB0063441E605F60012359
:105560009C46093BE2449C4674ABE3449B45C8D14E
:10557000029B9946A89B022B00DD82E0002B37DCC2
:105580001DD1059B00254B441E0000243268736822
:105590002800210001F038FB009B05000C00083EAC
:1055A0005A1E0092F2D2079B002B03D080231B06C9
:1055B0009C4664442A00230009990A604B60072036
:1055C0000B9B18409F239B009D443CBC90469946F2
:1055D000A246AB46F0BDC046FFFFFF3F0000F03FD4
:1055E0000000E03F0000703E00A60000FB21F93FF4
:1055F000059B00204B441E0000214CAF32687368AD
:10560000083E01F001FBBE42F8D1079B002B24D0DD
:105610008023099A1B06CB18106053600B00020010
:105620004E984F9902F0A4F9009B002B0BDD01244A
:1056300050AD0CCD01F0E8FA009B0134A342F8DA3A
:10564000079B002B03D080231B069C4661440B0064
:10565000020009998A60CB60B1E702000B00099C47
:10566000226063600B0002004E984F9902F080F9AF
:10567000009B002BDBDC0B00020009998A60CB60E9
:105680009DE7A89B032B9AD1009B002B00DCE3E055
:105690007E4A059B94464B441E685F68009B6344AA
:1056A0009A46DB004B4498464CAB9B4643465C68AD
:1056B0001B681800210032003B000290039101F0AA
:1056C000A3FA04000D0002000B000298039902F0F7
:1056D0004FF93B00320001F097FA43469860D960D9
:1056E0001C605D6008235B429C46E04426002F005E
:1056F000C345DBD1009B012B00DCADE0059BC84618
:105700004B441E685F685346DB009B46D8444346C3
:1057100030005C681B683900009301941A00230074
:1057200001F072FA04000D0002000B0000980199CC
:1057300002F01EF93B00320001F066FA4346986021
:10574000D9601C605D6008235B429C46E0442600F3
:105750002F00C145DBD15D460027002408354D44AC
:1057600050AE2A686B683800210001F04DFA083D00
:1057700007000C00AE42F4D1079B002B71D0099AB0
:105780004E994B461160802109068C465B6849465C
:10579000634453604B46DB688968634464449160AA
:1057A000D360176154610AE7994643460B93069B01
:1057B00030005A42390000F0BBF90022344B04009B
:1057C0000D0001F08FF8002832D0324B002220006B
:1057D000290001F053FE02F01FFC4A460600970024
:1057E00002F050FC00222A4B01F048FE02000B00A0
:1057F0002000290002F0BCF802F00EFC12AAD051E1
:105800004A46069B0132183300920693930012AA6F
:10581000D65044E601227FE500243AE5A89B022BFE
:1058200014DC002B0FDC00D0C9E600250024BAE60A
:105830004B46200029009E0002F0EEFB12AB98516F
:105840004B4600932BE600200021DEE64EAB994646
:10585000A89B032B00D0B2E6079B00270024002B57
:105860008DD14E9A4F9B09990A604B604B469A68BE
:10587000DB68009201938A60CB603A0023000A61E2
:105880004B619CE676AB0A9335E4C046FFFFFF1FF1
:10589000000070410000703EF0B54F464646C0B46F
:1058A00087B000920193464A4B00814688465B08C8
:1058B000934205DC02F0B0FB4146031E484666D029
:1058C0004A4643464846414601F0D8FD04000D00D3
:1058D00002000B004846414601F0D0FD394A3A4BE0
:1058E00006000F002000290001F0C8FD374A384BA0
:1058F00002F03EF822002B0001F0C0FD354A364B85
:1059000001F082F922002B0001F0B8FD334A344B3C
:1059100002F02EF822002B0001F0B0FD314B324A8C
:1059200001F072F90E9B02900391002B34D0009885
:10593000019900222D4B01F0A1FD029A039B0490D6
:1059400005913000390001F099FD02000B00049828
:10595000059902F00DF822002B0001F08FFD009A4E
:10596000019B02F005F8224A04000D00214B300093
:10597000390001F083FD02000B002000290001F036
:1059800043F902000B004846414601F0F1FF07B021
:105990000CBC90469946F0BD02000B002000290087
:1059A00001F06CFD124A134B01F0E2FF32003B00A4
:1059B00001F064FD4A46434601F026F9E7E7C04698
:1059C000FFFF3F3E7CD5CF5A3AD9E53DEB9C2B8A71
:1059D000E6E55A3E7DFEB157E31DC73ED561C119CC
:1059E000A0012A3F1111813FA6F810110000E03FED
:1059F000495555555555C53F49004B081900704745
:105A0000454AF8B5564692464B005B0D9A444D46C2
:105A10005F4644465246F0B4894605000C000E002D
:105A20000700132A22DC002A47DB52463B4B134176
:105A300098460B0042461340034311D0384A394B75
:105A400001F0E2F80022002300F042FF002805D018
:105A5000002C41DB4E46434600279E433800310070
:105A60003CBC90469946A246AB46F8BD5246332A06
:105A700008DD8023DB009A45F2D102000B0001F023
:105A8000C3F8EDE7284A9446012263445242DA40C3
:105A900093460242E4D0224A224B01F0B5F800229C
:105AA000002300F015FF0028D8D0002C1ADB5B463D
:105AB0004E469F4338003100D2E7194A194B01F096
:105AC000A3F80022002300F003FF0028C6D0002C1A
:105AD00016DB00270026C1E7802352465B031341F3
:105AE0009944B7E75346142B12D03423524601276A
:105AF0009B1A9F407F19AF429B415B429944D6E776
:105B00006400640825430027002DA7D0074EA5E7B1
:105B1000133B9C46E144CAE701FCFFFFFFFF0F0077
:105B20009C7500883CE4377EEDFBFFFF0000F0BF72
:105B30004B0070B55B0D14000A00002B1AD14B000E
:105B40005B08034315D00022224B01F097FC224B47
:105B50000A009C4222DB4B005B0D363B1F4DE318D5
:105B6000AB4220DC002B0DDD1D4C1B0522401A43EF
:105B7000110070BD1B4DAB42F0D102000B0001F0D3
:105B800043F8F6E71D00353518DA174B02009C4242
:105B90000ADC0B001548164900F032F8134A144B82
:105BA00001F06CFCE5E702000B001248124900F01E
:105BB00027F8104A104B01F061FCDAE7084C363345
:105BC00022401B051343190000220C4B01F056FC28
:105BD000CFE7C04600005043B03CFFFFFE07000087
:105BE000FFFF0F80FF07000050C3000059F3F8C209
:105BF0001F6EA5019C7500883CE4377E0000903C38
:105C000030B54A00DB0FDB0752081A43110030BDE4
:105C1000F7B506000D000C008B180193019B671B64
:105C20009C4207D0336821781B68300098470134C4
:105C30000028F3D13800FEBD70B505000C00081E29
:105C400007D002F089FF2B6802005B682100280062
:105C5000984770BD10B5FFF7EFFF10BD10B540229B
:105C60000021040002F04BFB002320002364636446
:105C700010BD3F23026C10B5541C2340446C9C4261
:105C800001D08154036410BD002303644364704752
:105C9000436C026C934206D03F21C25C01330B403F
:105CA0004364100001E0012040427047036C406CE7
:105CB000181A00D540307047436C026C934201D0F3
:105CC000C05C01E0012040427047036C406C5A1CEC
:105CD0003F231340181A42424241D0B2704700009D
:105CE00003210A4802680A430260094802680A431D
:105CF00002600849084A094B9B1A03DD043BC85857
:105D0000D050FBDC00F012F8FAF734FA240500401A
:105D100054050040D4A8000000000020A00200208C
:105D2000FEE7FEE7FEE7FEE7FEE7FEE72D4B10B5D8
:105D30001A78012A19D12C4A1268120715D12B4A58
:105D4000E0241168F0220800104021420BD12849BC
:105D50000968114209D12749274A11608021274A41
:105D60000902116001E03028F1D01A78012A0DD122
:105D70001D490968090709D1F0201C49096801403B
:105D8000402903D11A490968014223D01B68DBB2BC
:105D9000012B25D1144B1B681B0721D1134B1A680B
:105DA000F0231A40A02A04D1114A12681A4203D0E3
:105DB00016E0D02A14D1F7E7114B1A68012A03D153
:105DC000C022104B1A600BE00F4A1A601A68012AB1
:105DD000FCD1F5E7C1218020C900C0054250D5E7BC
:105DE00010BDC046E00F00F0E40F00F0E80F00F037
:105DF000EC0F00F0DFFF07C004050040186C004006
:105E000000EC064014EC064075930000012070473A
:105E100010B503681322DB69984710BD7047000076
:105E20000369054A9950FC331A6A002AFCD0002203
:105E300001201A627047C0461C050000030010B51F
:105E40005C331A781F2313400122110099400D4B37
:105E50000424D967C221036989005C505A60DA6062
:105E6000A0220021D20099500122074952425A50E3
:105E7000064914305A500C395A5008315A50FFF71D
:105E800003FF10BD04E100E00C0500001405000054
:105E900010B51430FFF70AFF10BD10B51430FFF72E
:105EA0000BFF10BD10B51430FFF7F2FE10BD00005F
:105EB000030070B55E331C780269604BD450030058
:105EC0005D331C785E4BD450030061331C785D4B0E
:105ED000012C0CD105005F352E78A225ED0056511E
:105EE000050060352E78A125ED00565100E0002414
:105EF000D4509623DB00994238D996231B0199424E
:105F000037D996235B01994236D996239B01994252
:105F100034D9E1239B01994232D99623DB0199427E
:105F200031D9E123DB0199422FD996231B029942F3
:105F30002DD9E1231B0299422BD996235B0299426A
:105F400029D9E1235B02994227D9E1239B02994297
:105F500025D93D4B994224D9E123DB02994223D92B
:105F6000E1231B03994221D8384B21E09E23DB0219
:105F70001EE09D231B031BE0354B19E0354B17E05A
:105F8000EC239B0314E0344B12E0344B10E0344B11
:105F90000EE0344B0CE0344B0AE0344B08E0344B59
:105FA00006E08023DB0403E0324B01E080235B0545
:105FB0003149002453500423243953501100FC313B
:105FC000CC600C62C1210134890014605C309460A3
:105FD000535003781F202200D9B2084082408034F9
:105FE0002648FF345BB20251002B13DA0F230B401B
:105FF000083B234C9B089B001B1903242140A14014
:10600000FC348C40DD69A543C0248C402100294329
:10601000D96111E0194C9B089B001B1903242140F6
:10602000A140C025FC348C40AD005E59A643C0247D
:106030008C40210031435951026070BD0C050000B5
:10604000140500006C05000090D0030000D0BE0EC7
:1060500000B013000050270000A04E0000F07500B3
:1060600000509D0000F0EB0000903A0100E0D701E5
:1060700000B0AF0300705F072405000000E100E0FE
:1060800000ED00E0F7B5009308AB1B780025019305
:10609000FA2304009B0083600E4B456008330360C5
:1060A00014300F001600FFF7D9FD23005C33276181
:1060B0001E70009B084A9B00995823005D3319709D
:1060C000019B20009B009A5823005E33DD701A70FC
:1060D000FEBDC04640A60000ECA30000036910B559
:1060E0001A00FC32D2680400002A0AD0A322D2008F
:1060F00099581430C9B2FFF7BCFD00222369FC3364
:10610000DA6010BD10B50248FFF7E8FF10BDC046C9
:10611000581100201D2307B50222009302490133C4
:106120000248FFF7AFFF07BD0020004058110020D4
:106130007047000010B500F011F8FFF7F9FF0120DB
:1061400000F0F0F9FEF7A2F9FEF7B4F9024B002BCC
:10615000FAD000E000BFF7E700000000C421114AB8
:1061600089005058104B0340C02000020343535095
:10617000802391399B02FF39535013608023A3225F
:106180000021DB05D20099500122A1209A60074B23
:10619000C0001950C1200231800019504030195000
:1061A0001A60704700E100E0FF00FFFF00100140AF
:1061B000014B18607047C046DC010020F7B5002392
:1061C0001E2877D83C4B8000C258042A14D006D829
:1061D000022A0DD00ED80423012A14D069E0062A21
:1061E0000ED00BD31A2A0DD002231B2A0BD060E04D
:1061F000082308E0102306E0202304E0402302E007
:10620000802300E001232D4A1268082A04D9092AB4
:1062100005D00A21022404E00821002401E0110035
:106220000124A02501261C272548ED004651254DB7
:10623000254E2D681B02AD003D400195234D2D6874
:1062400000958559AC466746214D3D401D4385511B
:106250008359C0259C46009BAD021D40FF23674625
:106260001B023B402B43019D1D43009B5F016023AC
:106270001F402B003B431C4301238451154C0360FA
:1062800063680F48002BFBD00024124B01255C6093
:10629000A123DB00C3584560A025ED0044511BB28B
:1062A000914207D002D98A1AD34003E0521A934090
:1062B00000E000231800FEBDECA30000E001002078
:1062C00000700040D801002004050000D401002027
:1062D000FF00FFFFFC700040F0B51E286CD8374B64
:1062E0008000C258364B1E68002E2ED1C22435487D
:1062F000A4000759344B03253B40C0273F023B43D2
:1063000003518023893C9B00FF3C03512F4F0360C6
:106310002F4B803CD859FF3CA043D8510437D85963
:10632000A8432043D8510837D8590C35A843083D15
:106330002843D851A820C0001E508026C1207602D4
:1063400080001E501C601E4B1C6000231426214838
:1063500034005C43255804006F1C0FD114205843AF
:106360002250A0200325C132FF329200C0051550F3
:10637000194A08001268082A03D10BE0AA4218D172
:10638000ECE7082A02D9083AD14002E00820821A34
:106390009140080014225343E3189A680C49513283
:1063A000FF32920058605050DA68C1239B00CA50F7
:1063B00002E00133032BCBD1F0BDC046ECA30000BB
:1063C000BC11002000E100E0FF00FFFF0405000019
:1063D00000900040E4010020DC0100201E4BF0B5DD
:1063E000596C18001D4A002914D0A025A1260023AD
:1063F0000124ED05F600D1584F1C06D0D7187F6850
:10640000002F02D027008F40AF5114333C2BF2D124
:1064100000234364131DA02540329446002001242C
:106420000F4EED05DA680F49920057180A495218C5
:10643000526C002A0CD01A1F1268511C05D0196822
:10644000FF2902D021009140A9513A00FC3250644A
:1064500014339C45E6D1F0BDFC900040E4010020DF
:106460000C0500000090004000B51E2816D80C4A0C
:1064700083009B58032911D8A0220800C133FF33A1
:10648000D2059B0000F06CF802080406002104E02D
:106490000C2102E0042100E00321D15000BDC046E0
:1064A000ECA300001E280DD8074B8000C058A02286
:1064B0000123D2058340002901D1044901E0A12133
:1064C000C90053507047C046ECA300000C05000003
:1064D000030000201E2B0AD8A222A021D200C90549
:1064E0008858034A9B009B58D840012318407047A6
:1064F000ECA30000084A0949094B10B51B688858ED
:10650000FA22190A1B0618439200002300F0F4F93E
:106510004904C00B084310BD0405000000100140F1
:10652000C011002070B5041E09D0FFF7E3FF05007D
:1065300000F014F8FFF7DEFF401B8442F8D870BD6E
:106540000022044B9A60044A13680133DBB21360E3
:106550007047C046FC100140C01100207047000089
:1065600002B4714649084900095C49008E4402BCE6
:106570007047C046002243088B4274D303098B4204
:106580005FD3030A8B4244D3030B8B4228D3030C03
:106590008B420DD3FF22090212BA030C8B4202D3A5
:1065A0001212090265D0030B8B4219D300E0090ACD
:1065B000C30B8B4201D3CB03C01A5241830B8B42D6
:1065C00001D38B03C01A5241430B8B4201D34B03BF
:1065D000C01A5241030B8B4201D30B03C01A524124
:1065E000C30A8B4201D3CB02C01A5241830A8B42A9
:1065F00001D38B02C01A5241430A8B4201D34B0292
:10660000C01A5241030A8B4201D30B02C01A5241F5
:10661000CDD2C3098B4201D3CB01C01A52418309A9
:106620008B4201D38B01C01A524143098B4201D3E3
:106630004B01C01A524103098B4201D30B01C01A0E
:106640005241C3088B4201D3CB00C01A5241830888
:106650008B4201D38B00C01A524143088B4201D3B5
:106660004B00C01A5241411A00D201465241104615
:106670007047FFE701B5002000F0F0F802BDC0460A
:106680000029F7D076E7704703460B437FD40022FA
:1066900043088B4274D303098B425FD3030A8B42B6
:1066A00044D3030B8B4228D3030C8B420DD3FF2220
:1066B000090212BA030C8B4202D31212090265D0EE
:1066C000030B8B4219D300E0090AC30B8B4201D3A1
:1066D000CB03C01A5241830B8B4201D38B03C01AE8
:1066E0005241430B8B4201D34B03C01A5241030B5F
:1066F0008B4201D30B03C01A5241C30A8B4201D310
:10670000CB02C01A5241830A8B4201D38B02C01ABA
:106710005241430A8B4201D34B02C01A5241030A31
:106720008B4201D30B02C01A5241CDD2C3098B4216
:1067300001D3CB01C01A524183098B4201D38B0193
:10674000C01A524143098B4201D34B01C01A524136
:1067500003098B4201D30B01C01A5241C3088B427B
:1067600001D3CB00C01A524183088B4201D38B0066
:10677000C01A524143088B4201D34B00C01A524108
:10678000411A00D201465241104670475DE0CA0FDF
:1067900000D04942031000D34042534000229C469F
:1067A00003098B422DD3030A8B4212D3FC228901A9
:1067B00012BA030A8B420CD3890192118B4208D37F
:1067C000890192118B4204D389013AD0921100E0E1
:1067D0008909C3098B4201D3CB01C01A52418309F5
:1067E0008B4201D38B01C01A524143098B4201D322
:1067F0004B01C01A524103098B4201D30B01C01A4D
:106800005241C3088B4201D3CB00C01A52418308C6
:106810008B4201D38B00C01A5241D9D243088B421C
:1068200001D34B00C01A5241411A00D201466346BF
:1068300052415B10104601D34042002B00D5494223
:10684000704763465B1000D3404201B5002000F062
:1068500005F802BD0029F8D016E770477047C0461A
:10686000D0400B1C1141203A03D49C4613411843DD
:1068700063465242934018437047C0468446101CFA
:1068800062468C46191C634600E0C0461FB500F006
:106890008BFD002801D40021C8421FBD10B500F0B7
:1068A000DFFC4042013010BD10B500F07DFD002836
:1068B00001DB002010BD012010BDC04610B500F066
:1068C00073FD002801DD002010BD012010BDC04671
:1068D00010B500F005FD002801DC002010BD0120EE
:1068E00010BDC04610B500F0FBFC002801DA002006
:1068F00010BD012010BDC046F0B54F464646C0B49D
:106900001604360C9946330005042C0C070C150CA4
:1069100063437E436F4365431C0CAD1964199C4669
:10692000A64203D980235B02984647446346250C60
:10693000EF191D044B464A4343432D0C24046419AC
:106940009918C91920000CBC90469946F0BDC04664
:10695000F0B557464E4645464300E0B446028846E9
:10696000760A1F0EC40F002F47D0FF2F25D000231B
:1069700080259A469946F600ED042E437F3F434614
:1069800042465D02D20F5B006D0A1B0E904640D05E
:10699000FF2B39D080220020ED00D20415437F3B2D
:1069A000FB1842465746591C62408C4607430F2F3E
:1069B0005CD86F49BF00C9598F46002E45D10823C6
:1069C0009A46063B9946DAE7424602282DD003282C
:1069D00000D1C3E0012800D0A2E00025002602403B
:1069E000D4B27602ED05760A2E43E4072643300042
:1069F0001CBC90469946A246F0BD002E1AD1042335
:106A00009A46033B9946BAE72A00511E8A41901CD8
:106A1000C6E70120002DC3D0280001F0C9FB431FA9
:106A200076309D4043420020BAE70124FF25144000
:106A30000026D6E7300001F0BBFB431F9E40002339
:106A4000763047429A46994699E70C239A46093B85
:106A5000994694E780260024F603FF25C1E7350018
:106A60004846B2E7350022004846AEE72904090C43
:106A70000800370C3604360C2C0C794370436743FE
:106A80007443060C64183619B14203D980214902B7
:106A9000884647440004000C310409188D01681E23
:106AA0008541890E2943350CED19AD010D432901AE
:106AB00004D5012369081D4063460D4319007F3149
:106AC000002925DD680704D00F202840042800D0C5
:106AD0000435280103D5274980330D401900FE29CC
:106AE000A3DC0124AD016E0A1440CDB279E7802009
:106AF000C003064207D0054205D128434602760A64
:106B00004446FF256DE706437602760AFF2568E7CF
:106B10000124611A1B2905DD14400025002660E7C9
:106B20006346CBE72E002023CE40591A8D406B1EC2
:106B30009D412E43730704D00F233340042B00D014
:106B40000436730104D5012401251440002648E7CA
:106B50000124B601760A1440002542E7802601246C
:106B6000F6032E437602760A1440FF2539E7C04625
:106B700070A60000FFFFFFF770B5002830D0C317E4
:106B8000C5185D40C40F280001F012FB9E231B1A9C
:106B9000962B0DDC9622D21A95406A02520AD8B280
:106BA0005202C005520AE40702432243100070BD9E
:106BB000992B19DC9922D21A9540124A2A4069076A
:106BC00004D00F210D40042D00D00432510103D513
:106BD0000C4B1A409F231B1A9201520AD8B2DFE7CE
:106BE000002400200022DBE705222E00121AB92122
:106BF000D6402A00C91A8A40551EAA4135001543BD
:106C0000DBE7C046FFFFFFFBF8B556465F464D4643
:106C10004446F0B40F00FD0FAA4609037C002E0085
:106C20005F00450F490A7F0D2943C5001803BC4684
:106C3000400A570F640DDB0F3843D2009A4500D14C
:106C4000AAE06646A61B002E00DCFFE06346002B90
:106C500039D10300134300D0D9E06B0709D00F23CB
:106C60002B40042B05D02B1DAB42AD416D42491981
:106C70001D000B0200D482E0CA4B01349C4200D1BB
:106C8000FEE00A005646C84BED081A40500764055E
:106C900052020543120B640D002112030B0D1B055C
:106CA0006405120B1A436308C04CF60714401C43DA
:106CB000640064083443280021003CBC9046994697
:106CC000A246AB46F8BDB74B9C42C6D080231B04FE
:106CD0001843382E00DDEBE01F2E00DD1EE12023DF
:106CE0009B1B9C4603006746BB40984613004746E3
:106CF000F3403B436746BA40571EBA411343020074
:106D0000F240EB1A9D42B6411D008A1A7642911B51
:106D10000B0231D54A02560A002E00D1B4E03000F1
:106D200001F046FA0300083B1F2B00DDB5E02022EE
:106D30002900D21AD1409E400A009D4032439C4215
:106D400000DDB1E01C1B631C1F2B00DDD5E0202102
:106D500014002800C91A8C40D8408D400443DA4002
:106D6000681E854111002543002476E741463143E2
:106D700000D134E2310045466B0700D06FE756463C
:106D80004807ED08C9080543864B9C4235D00A03E5
:106D90006405120B640D7FE76346E31A9B46002BE4
:106DA00000DC8BE06746002F3CD07E4FBC4200D118
:106DB00053E780273F0438435B46382B00DCF7E07D
:106DC0000243501E82410020D2B253194218AB42F6
:106DD00089411D00494289180B02CDD5714B013400
:106DE0009C4200D13DE101206F4A6B080A402840D7
:106DF0001843D507054351082FE72B000B4300D15B
:106E0000CBE180231B030B431A03120B44E7013E23
:106E1000002E6DD1AE1AB5429B41091A5B42C91AC8
:106E2000350075E70700174300D116E701235B42E1
:106E30009C46E3445B46002B00D0E0E0AA18AA423F
:106E40009B4109185B4259181500C5E7002E75D102
:106E5000661C7605760D012E00DCF3E0AE1AB04616
:106E60004545BF410E1A7F42F61B370200D48FE022
:106E7000551BAA42B641411A76428E1B9A464BE7F1
:106E800056460022002507E7280001F091F920303E
:106E90000300083B1F2B00DC49E72A00283882400A
:106EA00000259C4200DC4DE73F49E41A1140D4E63E
:106EB0000243501E8241D3B2002222E7002B00D0B1
:106EC000F3E0631C9C465B055B0D012B00DC9FE03F
:106ED000344B9C4500D1C3E0AA180918AA4280414E
:106EE00040424118CD075208154349086446B4E6AC
:106EF0002C4B9C4200D0ECE6AFE611001F3CE14079
:106F00000C00202B00D17FE04021CB1A9A40154382
:106F10006A1E95410021254300242DE73300070018
:106F2000203BDF403B00202E70D04027BE1BB040EE
:106F30000243501E824113430022E2E6002C4FD050
:106F4000184CA44500D1ABE08024240476422143B0
:106F5000382E00DDDFE01F2E00DD43E12027BC1BC3
:106F6000A1460C004F46BC40A0462C004746F440CA
:106F70003C434F46BD406F1EBD41F1402C43151BA5
:106F8000AA429241411A5242891A64469A46BFE681
:106F900041464546314300D0BEE600260024002588
:106FA000F2E6C046FF070000FFFF7FFFFFFF0F80F4
:106FB0001F2B59DC2027FF1ABC46070063469F4061
:106FC0005B46B9461700DF40B8464F4643461F436D
:106FD00063469A40531E9A415B463A43D840F4E6D2
:106FE0000C002C435CD0F643002E55D1551BAA4211
:106FF000A441411A6442091B9A46644688E6964FAA
:10700000BC4200D0D8E628E6002280E700208FE7C7
:107010000B002B43002C00D0C2E0002B00D101E17B
:107020000300134300D118E6AB18AB42B641091870
:10703000764271180A0200D409E1884A1D00114005
:1070400064460AE6002C5BD10E002E4300D08AE095
:107050000100114300D1C2E0010015009A46FCE591
:107060006446002100258FE620235B429C46DC44D9
:1070700063460700DF405B46BC46202B00D1ACE0F6
:1070800040235F46DB1B98400243501E824163460B
:1070900013431A00002098E66F4CA44500D057E730
:1070A0000100150064469A46D7E5002C39D10C0042
:1070B0002C436ED0DB43002B1AD0674CA44568D01C
:1070C000382B00DDA4E01F2B00DDAEE020240F00F4
:1070D000E41AA740B9462F00DF40B846A3464F4602
:1070E000444627435C46A5406C1EA541D9403D431C
:1070F000AD1895429B4109185B42591864466BE6EE
:107100000C002C4315D1010011437BD00100150068
:107110009A46514CA1E50D43691E8D410021ECB208
:107120002DE74D4CA44534D0802424045B422143F8
:10713000C6E7040014434ED0ED084C072C438025CD
:10714000C9082D03294208D0C6082E4205D1D2080D
:10715000410711430C009A463100620FC900E50057
:1071600011433D4C79E50600164300D175E5AE1A92
:10717000B0464545BF410E1A7F42F61B370200D488
:10718000F4E5551BAA42B641411A7642891B9A463C
:1071900063E50100150064465FE5002200257BE5FC
:1071A000002B3BD00300134315D0ED084B072B43B6
:1071B0008025C9082D03294207D0C4082C4204D1D8
:1071C00041070B002100D2081343C9005A0F114395
:1071D000DD00214C41E5204C3FE5002054E700262E
:1071E0000025D1E534000F00203CE7403C00202E74
:1071F0002BD04027BE1BB1400D43691E8D4100219D
:107200002C43BCE6802100260903134C0025BBE576
:107210000D43691E8D410021EDB269E701001500A3
:107220000D4C1AE50100150017E51C000F00203C6D
:10723000E7403C00202B0CD04027FB1A99400D431F
:10724000691E8D410021254352E70021D4E71D002E
:1072500092E50021F3E7C046FF070000FFFF7FFF34
:10726000F0B55F4656464D464446F0B41F035C00F9
:10727000DB0F9A46194B0E034D00C90F8046360BA3
:107280006D0D8B4691463F0B640D9D4219D0134BFB
:107290009C421BD00123A54206D018003CBC90465E
:1072A0009946A246AB46F0BDBE42F6D1C845F4D1E0
:1072B000D34510D0002DF0D1304303005A1E934126
:1072C000EBE7310001230143E7D1E0E73A43012333
:1072D000002AE2D1DEE70023DFE7C046FF07000017
:1072E000F0B55F46444656464D46F0B41F033C0B8E
:1072F0002C4F0E034D00A3465C008446360B6D0DEB
:10730000C90F9046640DDB0FBD422BD0254FBC4208
:107310002ED0002D0ED130430700814678427841AF
:10732000002C17D15F463A4314D14B460020002B66
:107330000AD006E0002C02D15846024301D09942FF
:107340001AD00123484218433CBC90469946A246B5
:10735000AB46F0BD0028F2D05842584101224042CD
:107360001043F1E737000743D0D002204042EBE75B
:107370005F461743CDD0F8E7A542E2DC05DB5E456A
:10738000DFD808D000205E45DED2484248410123C4
:1073900040421843D8E7C445D3D80020C445F4D3AD
:1073A000D2E7C046FF070000F0B55F464D464446B1
:1073B0005646F0B41C03240BA4462F4C0F034D007B
:1073C0005E00C90F80463F0B6D0D8B469146760DD2
:1073D000DB0FA54220D0284CA64222D0002D12D18E
:1073E000384344424441002E20D0002C0DD05C4252
:1073F000634101245B421C4320003CBC90469946FB
:10740000A246AB46F0BD002E17D05B4519D05B46B7
:107410005C4201231C43EFE7390002240143EBD116
:10742000D9E7614602241143E6D1D7E761460A4312
:10743000DBD100240028DFD0E9E761460A43E4D12C
:10744000E5E7B54203DD01225C421443D4E7B542CF
:10745000CDDB6745DBD809D000246745CCD259463F
:107460004C426141012449420C43C5E7C845CED88E
:107470000024C845F3D3BFE7FF070000F0B55F461F
:1074800056464D464446F0B40D0399464E002B0B2C
:1074900087B00700924680469B46760DCC0F002EA3
:1074A00069D06D4B9E4235D05B468022DD001204D0
:1074B000430F13432B439B46C3009846674B00275B
:1074C0009C460023664401934A4615035000D20FA0
:1074D00053462D0B400D914600D176E05E4A904216
:1074E0006CD080225B0F120413435C4AED0094467B
:1074F0001D4353460022DB00604449463618701C89
:107500006140029017430F2F00D9AFE05448BF00ED
:10751000C759BF465B461F4300D088E000239B4607
:107520009846023308270193CEE74946022A6AD0DB
:10753000032A00D109E2012A00D0BBE11140002258
:10754000002300259046CCB200212D030A0D120520
:107550002D0B1543434A1B0515401D436D00E407E1
:107560006D0825434046290007B03CBC904699462B
:10757000A246AB46F0BD034352D05B46002B00D180
:107580008AE1584600F014FE03000B3B1C2B00DD83
:107590007BE11D22D31A3A0001005D46DA4008392A
:1075A0008D4013008F402B439B46B8462E4B00273F
:1075B0009C46002360444642019385E752462A4395
:1075C0002CD100250023022297E752462A4321D0DE
:1075D000002D00D154E1280000F0EAFD03000B3B30
:1075E0001C2B00DD46E11D21CB1A51460200D9407B
:1075F0005346083A954093400D431B4A94466044D5
:107600004042002279E7012400220C40124B002561
:10761000904699E70025002301226EE703226CE7DC
:1076200000239B4698460133042701934CE703232C
:107630000C27019348E700238025984600242D035A
:10764000054B81E75D464346019A6FE75D46434639
:107650002100019A6AE7C046FF07000001FCFFFF16
:10766000B0A60000FFFF0F80F30300004246120C9B
:1076700091461A0C9446424617044A461B041B0CBA
:107680005A43604690464A4642431000039262467F
:107690001C003F0C7A437C4342440192220C9246E8
:1076A000019A5244904506D9824680204002804685
:1076B000C24450460390100C049048462404240C05
:1076C0001204121905922A0C2D042D0C68432C006B
:1076D000824648467C4350438146200C80465743AF
:1076E00057444744BA4503D9802040028046C144EC
:1076F000380C3F04B84648442404240C01900498F4
:10770000A044404404905846000C81465846040466
:10771000200C8246070048465F434C464343604680
:1077200060436446834650464443380C8446E4181C
:107730006444A34203D980235B029C46E344484649
:107740003F04230C3F0C2404E419574668436F435D
:1077500084464D46504655434243380C8146624468
:107760004A445B44944503D98020400284466544E2
:1077700003983F04834604983F0C8446E344C34582
:107780008041404282461004844601986744844602
:107790006744A344BC46A345A4419946D4446442EB
:1077A0008742BF41D4458041E144A04699459B4171
:1077B0007F424042C8440743120CBA18A045A44176
:1077C0005F423B0064422343D71843467D19DB0DDB
:1077D0006D021D435B465A02059B1A43531E9A4194
:1077E0005B46DB0D1A4343465B021343EA0107D5B0
:1077F00001225C0813402343EA07029E13436D08ED
:10780000574AB218002A4BDD580709D00F201840FC
:10781000042805D0181D98429B415B42ED180300D7
:10782000E80104D54F4A15408022D200B2184E48D4
:10783000824200DDE7E60124DB08680718436D0299
:10784000530580462D0B5B0D0C407DE6802259468A
:107850001203114208D0154206D115432D03984654
:107860002D0B4C46414B6FE65D4615432D032D0B0A
:107870003E4B69E603005546283B9D400023BCE68D
:10788000504600F095FC2030A8E60300283B9F40BE
:107890000023BB46984689E600F08AFC203073E658
:1078A0000124A61A382E07DD00220C4000230025F3
:1078B000904649E6029EA3E71F2E20DC20222C00E2
:1078C0001800921BF040944093400443581E83419B
:1078D0001C43F540630709D00F232340042B05D038
:1078E00023001C1D9C4292415242AD182B021FD511
:1078F000012400220C4001230025904624E61F208D
:107900002C004042821AD440202E1CD04022961BCC
:10791000B5402B43581E83410720234318400025C0
:10792000002809D00F2200251A401C00042AD8D1B3
:10793000230068076D022D0B0124DB0803439846E2
:107940000C40002300E60025E3E780220124120317
:1079500015432D0398462D0B0C40044BF4E5C0460F
:10796000FF030000FFFFFFFEFE070000FF0700000F
:10797000F0B557464E464546E0B40E001100F20FF2
:107980009246C500420F180337037400400A4E0F99
:107990007F0A3043CF4E17435A00640D520DDB0F60
:1079A000C900B24200D1E5E001267340A61AB446F0
:1079B000534500D1AFE0002E00DC0DE1002A3AD1A2
:1079C00003000B4300D0E4E06B0709D00F232B40EA
:1079D000042B05D02B1DAB42AD416D427F191D001C
:1079E0003B0200D488E0BB4B01349C4200D110E143
:1079F0003A00B94B51461A4001235007ED08520294
:107A000064050543120B640D0B400021280012038E
:107A10000D0D120B64052D0515436208AF4CDB07F5
:107A20002C401443640064081C4321001CBC904695
:107A30009946A246F0BDA74B9C42C5D080231B04AB
:107A400018436346382B00DDFDE01F2B00DD30E1DD
:107A5000624620239B1A02009A40664690460A001E
:107A60009940F24046464B1E9941324311436346CA
:107A70000200DA40691A8D429B410D00BA1A5B423E
:107A8000D71A3B0235D57A02530A98464346002B53
:107A900000D1C4E0404600F08BFB0300083B1F2BE5
:107AA00000DDC5E020222900D21A4746D1409F4080
:107AB0000A009D403A439C4200DDC0E01C1B631C51
:107AC0001F2B00DDE4E0202114002800C91AD84053
:107AD0008C408D400443DA40681E854117002543E1
:107AE000002471E7424663461A4300D14CE26746E0
:107AF00045466B0700D069E7012351467807ED083A
:107B0000FA080B40054373498C4238D012036405D0
:107B1000120B640D79E7002E00DC9AE0002A47D0B2
:107B20006C4A944200D14FE780221204104362460F
:107B3000382A00DC08E10143481E81410022C9B215
:107B40004919D219A942BF410D007F42BF183A021C
:107B500000D442E15F4A0134944200D14EE1012059
:107B60005D4A69083A4028400843D507054357084D
:107B70009A4629E706000E4300D017E714E72900CC
:107B8000114300D1F9E1802109030A431203120BCA
:107B90003BE701235B429846C4446346002B72D105
:107BA000691A8D429B413F1A5B42FF1A0D0068E73C
:107BB00002000A4300D107E7012252429046C44422
:107BC0006246002A00D0E6E06918A942B6413F1893
:107BD0007642F7190D00BAE7002E00D080E0621C53
:107BE0005205520D012A00DCF9E06A1A91464D4512
:107BF000B6413A1A7642921B9046120200D499E09E
:107C00004D1BA9428941C71B49427A1A90469A46A0
:107C10003CE752460123002513400022F5E62800E8
:107C200000F0C6FA20300300083B1F2B00DC39E7C8
:107C30002A002838824000259C4200DC3EE7264F7F
:107C4000E41A1740C0E60143481E81410022C9B230
:107C500010E7002E00D0F1E0621C94465205520D50
:107C6000012A00DCA0E01B4A944500D1C5E0691858
:107C7000A94292413F185242D2194908D5070D43F3
:107C800057086446A0E6134B9C4200D0D9E69BE619
:107C900011001F3CE1400C00202B00D180E040216E
:107CA000CB1A9A4015436A1E9541002725430024AC
:107CB0001FE763460200203BDA406346202B71D069
:107CC000402366469B1B98400143481E8141114357
:107CD0000022CFE6FF070000FFFF7FFFFFFF0F80BE
:107CE000002C48D0CA4CA24200D1A2E07442A14666
:107CF0008024240427434C46382C00DDDBE01F2C75
:107D000000DD44E14E462024A41B3E00A640A246CE
:107D1000B0464C462E00E640B446464664462643EE
:107D20005446A5406C1EA54134002C434D46EF40FF
:107D30000D1B28E04A4643464D461A4300D0A5E6AF
:107D4000002300240025DEE61F2A5ADC6646202296
:107D5000921B060096409146B04662460E00D64001
:107D6000424616434A4691404A1E914102006046EF
:107D70003143C240E4E63C002C435AD0F443A146D0
:107D8000002C52D14D1BA9428941C71B49427F1A81
:107D900014009A4675E69E4A944200D0C7E613E660
:107DA00000227FE700208FE7002C00D0C8E03B00D6
:107DB0002B4300D10FE103000B4300D104E6691807
:107DC000A9429B413F185B42DF193B0200D41AE1F4
:107DD000904B0D001F406446F6E59A4689E63A004E
:107DE0002A43002C5CD1002A75D102000A4300D13D
:107DF000CAE007000D009A46E6E564460022002529
:107E000081E662460600203AD6406246B046202A05
:107E100000D1B7E040226646921B904001434246A3
:107E2000481E8141114300228AE6794CA24200D0CB
:107E300061E707000D0014009A46C5E5002C41D10A
:107E40003C002C4378D0F443A146002C20D0704C49
:107E5000A24271D04C46382C00DDB2E01F2C00DD70
:107E6000BCE02026341BA2463C005646B4404E4699
:107E7000A0462C00F440A446444666463443A4463B
:107E80005446A54064466E1EB54125434C46E74026
:107E90006D188D4289413F184942CF19140056E6AA
:107EA000002A2FD102000A4300D184E007000D0010
:107EB0009A46574C88E53D436F1EBD41ECB2002702
:107EC0000D1B60E7524CA24236D074428026360425
:107ED000A1463743BEE702000A4300D174E56A1A9F
:107EE00090464545B6413A1A7642921B9446120294
:107EF00000D4F7E54D1BA9428941C71B49427F1AAF
:107F00009A4661E502000A433AD0ED087C072C430B
:107F10008025FA082D032A4208D0C7082F4205D130
:107F200045072C003A009A46C9080C43670FD20057
:107F3000E5001743364C47E507000D00140043E504
:107F40003A002A4343D002000A4319D0ED087C07C7
:107F50002C438025FA082D032A4207D0C6082E425A
:107F600004D147073C003200C9080C43D700620F18
:107F7000E50017439A46264C26E50022002544E5F5
:107F8000234C21E5002049E700230025BBE54C46B2
:107F90003E00203CE6404C46B446202C31D04024E4
:107FA0004E46A61BB7403D436C1EA54164462C437C
:107FB00000270D1BE7E6802200231203144C002546
:107FC000A1E53D436F1EBD410027EDB260E707000C
:107FD0000D000F4CF8E407000D00F5E44E463C00A0
:107FE000203EF440A0464C46202C0ED040244E4665
:107FF000A41BA7403D436F1EBD41444600272543B7
:1080000046E70027CFE70D0073E50027F2E7C046FB
:10801000FF070000FFFF7FFF0B0330B5134D1A0B66
:108020004B005B0DC90F0024AB4211DD104CA34285
:1080300010DC8024640322430E4CE41A1F2C0CDD58
:108040000D48C31ADA4013005C42002900D11C001D
:10805000200030BD094BCC18FAE7E040084CA4469C
:1080600063449A4013000343EEE7C046FE0300005A
:108070001D0400003304000013040000FFFFFF7F15
:10808000EDFBFFFF70B5002830D0C317C4185C406B
:10809000C50F200000F08CF8174B184A1B1AD21A93
:1080A0001F2A18DD164AD21A9440002224035B05C9
:1080B000240B5B0D0021100024030A0D1205240B74
:1080C0001443104A1B0514401C436400ED07640868
:1080D0002C43210070BD210091400A000B21081A99
:1080E000C4405B052403240B5B0DE3E7002500235C
:1080F00000240022DEE7C0461E0400003304000016
:1081000013040000FFFF0F804200120E511C4302B7
:10811000C9B270B55D0AC40F012915DDE0218900DF
:108120008C466D071B0B6244002128000D0D2D05A8
:108130002B431C4D52052B40520813435B00E407B0
:108140005B082343190070BD002A15D1002D1FD0F4
:10815000280000F02DF80A281DDC0B232A001B1A2A
:10816000DA4013000200153295400F4A1B03121A21
:1081700052051B0B520DD7E7002D06D080221B0B9A
:10818000120313436D07094ACEE7084A0023CBE7E1
:1081900000220023C8E703000B3B9D402B00002575
:1081A000E3E7C046FFFF0F8089030000FF070000E0
:1081B0001C2101231B04984201D3000C10391B0A17
:1081C000984201D3000A08391B09984201D30009DB
:1081D000043902A2105C40187047C0460403020232
:1081E0000101010100000000000000007FB51D003A
:1081F0000A4B06001B68D868002A02D1084C2300ED
:1082000001E01300074C0293009133002A00064955
:10821000019400F021F800F023FEC0468002002007
:10822000B6A00000F0A60000FDA60000084B10B5A7
:108230000400002B02D0002100E000BF054B1868AD
:10824000836A002B00D09847200001F0F3FAC04663
:108250000000000030A700000EB403B5010003AB1E
:10826000044804CB0068019300F016F902B008BC82
:1082700003B01847800200200E4B70B500251E0089
:108280000D4CE41AA410A54204D0AB00F358984753
:108290000135F8E701F0D0FA084B00251E00084C24
:1082A000E41AA410A54204D0AB00F3589847013556
:1082B000F8E770BD880200208802002088020020B4
:1082C0009802002010B5034B0100186800F066F812
:1082D00010BDC0468002002010B5034B0100186895
:1082E00000F016F810BDC04680020020002310B533
:1082F0009A4203D0CC5CC4540133F9E710BD0300AB
:108300008218934202D019700133FAE770470000D7
:1083100030B500293ED004390B68002B00DAC918AB
:108320001D4A13681400002B02D14B60116031E02C
:108330008B420DD90A688818834203D118685B689C
:1083400082180A604B60216024E08A4203D813003F
:108350005A68002AF9D11D685C198C420BD1096852
:10836000691858181960824214D11068526841186F
:1083700019605A600EE08C4202D90C23036009E0B8
:1083800008680C18A24203D11468526820180860CB
:108390004A60596030BDC046C8110020032370B543
:1083A000CD1C9D43083506000C2D01D20C2505E09F
:1083B000002D03DA0C230020336040E0A942F9D8F5
:1083C0001F4B1C681A002100002913D00B685B1B8F
:1083D0000DD40B2B02D90B60CC181EE08C4202D1BD
:1083E000636813601AE04B6863600C0016E00C00D1
:1083F0004968E9E7134C2368002B03D1300000F0F3
:1084000033FB20602900300000F02EFB431CD1D04C
:108410000323C41C9C43A0420AD1256020000722EC
:108420000B30231D9043C31A09D05A42E25006E094
:10843000211A300000F018FB431CEED1BAE770BDE2
:10844000C8110020C4110020936810B5013B93604F
:10845000002B05DA9469A34208DBCBB20A2B05D0C6
:108460001368581C10601970C8B201E000F02CFCB1
:1084700010BDF8B506000F001400D518AC4208D0A6
:1084800021783A003000FFF7DFFF0134431CF5D1BB
:1084900000E00020F8BD0000F0B59FB006000F001E
:1084A00002920593002804D08369002B01D100F0CB
:1084B000D3FD7F4B9F4201D1776808E07D4B9F42FF
:1084C00001D1B76803E07C4B9F4200D1F768BB89BC
:1084D0001B070AD53B69002B07D0002306AD6B6153
:1084E00020336B761033AB763DE03900300000F07E
:1084F00043FC0028F1D001204042D6E0059A111D2E
:1085000012680591002A00DA7FE00992013423788D
:108510002E2B00D18DE021780322684800F082FEE6
:10852000002807D0654B2A68C01A402383401343B4
:108530002B6001342178631C06226148029329765E
:1085400000F070FE002800D19DE05E4B002B00D0B3
:1085500090E00722059B07339343083305936B692B
:10856000039A9B186B61029C2378002B04D1029B19
:10857000E31A049312D003E0252BF8D00134F3E77B
:10858000049B029A39003000FFF773FF431C00D1AF
:1085900086E06A69049B944663446B612378002BF0
:1085A0007ED00122002352426A6002A9543252183E
:1085B00001342B60EB60AB601370AB652178052252
:1085C000414800F02FFE002808D03F4B2A68C01A0F
:1085D0000123834013432B600134EFE72B68DA0655
:1085E00004D55322202102A8121811701A0704D5AD
:1085F00053222B2102A81218117022782A2A00D1A6
:108600007CE7099B00200A2105E05242EA60022231
:1086100013432B607AE72278303A092A04D84B4377
:1086200001349B180120F6E7002800D16FE7099379
:108630006DE763782A2B0AD1059B02341A1D1B684B
:108640000592002B01DA01235B42079363E70023C5
:108650000A201A0001346B6021783039092904D8C6
:108660004243013452180123F6E7002B00D152E7B0
:10867000079250E705AB00933A00144B29003000F5
:1086800000E000BF07E005AB00933A000F4B290064
:10869000300000F08BF80390039B013300D05EE7BD
:1086A000BB895B0600D526E70B981FB0F0BDC0461E
:1086B00068A8000088A80000A8A800003AA7000049
:1086C0003EA700000000000034A7000073840000F3
:1086D000F7B5170001938A680B6900900C0093426C
:1086E00000DA130022003B6043321278002A01D0E6
:1086F00001333B6023689B0602D53B6802333B6035
:10870000062523681D401ED0230043331B785A1EC4
:108710009341226892061CD53020E118433108703D
:1087200021005A1C45310978A218433202331170D6
:108730000FE022000123193201990098089EB047EA
:10874000431C0ED00135E3683A689B1A9D42F0DB6A
:10875000DAE72200019943320098089DA847431C9C
:1087600002D10120404220E006232068E1683A68F7
:1087700003400025042B03D18D1AEB43DB171D406A
:10878000A3682269934201DD9B1AED180027BD42C0
:108790000AD0220001231A3201990098089EB0479E
:1087A000431CDED00137F2E70020FEBDF0B58BB0F0
:1087B00006920A0043320793059004920A7E0C0049
:1087C000109B6E2A00D1ABE011D8632A22D009D8C1
:1087D000002A00D1B5E0582A00D0C5E045310A7022
:1087E000814A4FE0642A1DD0692A1BD0BCE0732A5D
:1087F00000D1AAE009D86F2A29D0702A00D0B3E0AE
:10880000202209680A43226037E0752A1FD0782A9F
:1088100033D0A9E00E001A684236111D19601368A2
:108820003370A4E021681A68080606D4490604D506
:10883000111D19600023D55E02E0111D1960156835
:10884000002D3BDA2D23049A6D42137036E0216827
:108850001A68080606D4490604D51568111D196062
:10886000ADB202E0111D196015685F4B227E0393C3
:1088700008276F2A1DD00A271BE0220078214532E5
:1088800011705A4A19680392081D226818600D6811
:10889000100602D4500600D5ADB2D30702D520236E
:1088A0001A4322601027002D03D1202322689A4307
:1088B00022602300002243331A7002E00A274A4B49
:1088C00003936368A360002B09DB042221689143B2
:1088D0002160002D05D1049E002B11D07BE0002DDE
:1088E00079D0049E28003900FDF7CAFE039B013EA3
:1088F0005B5C280033703900FDF73CFE051EF1D1AA
:10890000082F09D12368DB0706D5636822699342E3
:1089100002DC3023013E3370049B9B1B23612BE060
:1089200009681A68080607D4490605D5111D19609B
:108930001368A28A1A8004E0111D19601368626925
:108940001A600023049E236116E01A68111D196045
:10895000166800216268300000F064FC002801D035
:10896000801B6060636803E026004236327001239A
:1089700023610023049A1370079B09AA0093210026
:10898000069B0598FFF7A4FE431C02D1012040423C
:1089900027E02369320006990598079DA847431CE4
:1089A000F4D0236800259B070FD4099BE068984208
:1089B00017DA180015E022000123193206990598EC
:1089C000079EB047431CE1D00135E368099A9B1A22
:1089D0009D42F0DBE9E72600039B42361B783370AB
:1089E0008EE70BB0F0BDC04645A7000056A70000BB
:1089F000154B10B51C68A36B002B15D11820FFF781
:108A000061FC124BA0630380114B01224380114B88
:108A10008380114BC380114B0381052343810633AF
:108A20008381002302614361A46B0D4A206961695F
:108A30000C4BFDF761FF0122002380185941206192
:108A400061614800400810BD800200200E33000024
:108A5000CDABFFFF341200006DE6FFFFECDEFFFF41
:108A60002D7F954C2DF45158002370B5064C050010
:108A70000800236000F0C8FE431C03D12368002BCC
:108A800000D02B6070BDC046E02500200CB430B58E
:108A9000164B9DB00C1E1D6804DA8B2301202B6041
:108AA00040421DE0822302A99B008B81002302909B
:108AB00008619C4200D0631E8B604B6101235B42C6
:108AC000CB81209A21AB2800019300F053FC431C7A
:108AD00001DA8B232B60002C02D00023029A137042
:108AE0001DB030BC08BC02B01847C0468002002050
:108AF0000EB410B59DB002A9029008610B48822403
:108B000088604861012040421FABC881084804CBFF
:108B1000A400006801938C8100F02CFC0023029AD1
:108B200013701DB010BC08BC03B01847FFFFFF7FD7
:108B30008002002002780B78002A03D00130013136
:108B40009A42F7D0D01A7047031C0A7801311A7084
:108B50000133002AF9D170470023C25C0133002A97
:108B6000FBD1581E7047030030B5002A0DD00C7899
:108B700001335D1E013A2C700131002CF5D19A1899
:108B80009A4202D01C700133FAE730BDF0B51E00E6
:108B9000454B87B01B680192029308220B00059099
:108BA00003911C7802995D1C09194878104001D086
:108BB0002B00F6E72D2C04D19D1C5C78012300933B
:108BC00004E000902B2C01D15C789D1C002E02D07B
:108BD000102E0AD162E0302C5ED120222B789343F4
:108BE000582B54D110266C780235009F31007B1E23
:108BF0009F412E4BFF183800FDF742FD38000491CD
:108C00003100FDF7B7FC002303220700944618004B
:108C1000029A121951780422114201D0303C07E027
:108C20006246114017D03722012900D02032A41A01
:108C3000A64210DD5A1C0BD0B84207D802D1049BC3
:108C40009C4203DC70430123201801E001235B42B6
:108C50002C780135DCE75A1C0BD10098059A431E8D
:108C60009841124BC01822231360019B002B0AD19C
:108C700017E0009A002A00D04042019A002A10D042
:108C8000039A002B00D06A1E019B1A6009E0302471
:108C9000002EAAD10826A8E70A26A6E7302C9CD0E9
:108CA000A3E707B0F0BDC04684020020FFFFFF7FAE
:108CB00010B513000A00010002480068FFF766FFC4
:108CC00010BDC04680020020F8B505000F0014005A
:108CD000002804D08369002B01D100F0BDF9234B9B
:108CE0009C4201D16C6808E0214B9C4201D1AC68E8
:108CF00003E0204B9C4200D1EC68A369A360A389E8
:108D00001B070AD52369002B07D023682269FEB20E
:108D1000981A636998420FDB08E02100280000F0F0
:108D20002BF80028F1D0012040421DE0210028004E
:108D300000F024F90028F6D1A3680130013BA360BC
:108D400023685A1C22601F706369984205D0A3896A
:108D50003000DB0708D50A2E06D12100280000F0DC
:108D60000DF90028DFD13000F8BDC04668A800002A
:108D700088A80000A8A80000354B70B51D68060043
:108D80000C00002D05D0AB69002B02D1280000F0AB
:108D900063F9304B9C4201D16C6808E02E4B9C4239
:108DA00001D1AC6803E02D4B9C4200D1EC68A38953
:108DB0009AB2110723D4D10607D4092201203260C8
:108DC00037321343A381404240E0530713D5616B10
:108DD000002908D023004433994202D03000FFF725
:108DE00097FA002363632422A3899343A38100237A
:108DF0006360236923600822A3891343A381236945
:108E0000002B0BD1A023A2899B001340802292004B
:108E1000934203D02100300000F0B2F90123A2896F
:108E2000134005D00023A36063695B42A36103E0A4
:108E3000910700D46369A36000202369834205D1B0
:108E4000130603D540231A43A281013870BDC046E2
:108E50008002002068A8000088A80000A8A80000E0
:108E600010B5062000F0AEFB012000F0E3FC00008E
:108E7000F7B58A8905000C0013075AD44B68002BFC
:108E800002DC0B6C002B19DDE76A002F16D00023E3
:108E90002E682B6080235B011A4001D0606D14E0C6
:108EA0000123216A2800B847431C0ED12B68002BF0
:108EB0000BD01D2B01D0162B02D12E6000205AE0C2
:108EC0004022A3891343A38155E0A3895B0706D5FC
:108ED0006368C01A636B002B01D0236CC01A002397
:108EE0000200216A2800E76AB847A389421C06D11C
:108EF00029681D293AD8204ACA40D20736D500220F
:108F0000626022692260DB0405D5431C02D12B6814
:108F1000002B00D16065616B2E600029CED023004C
:108F20004433994202D02800FFF7F2F90020606331
:108F300021E00F69002FC1D00B680F60DB1B01938C
:108F40000023920700D14B69A36003E0019B3F1807
:108F50001B1A0193019B002BB0DD019B3A00216A93
:108F60002800A66AB0470028F0DCA389402201202F
:108F70001343A3814042FEBD010040200B6970B540
:108F800005000C00002B01D100201CE0002804D0BB
:108F90008369002B01D100F05FF80B4B9C4201D19B
:108FA0006C6808E0094B9C4201D1AC6803E0084BB7
:108FB0009C4200D1EC680C22A35E002BE4D021007F
:108FC0002800FFF755FF70BD68A8000088A80000C2
:108FD000A8A8000010B5024900F0B0F810BDC046C6
:108FE0007D8F0000002310B50400036043608360A0
:108FF00081814366C2810361436183611900082254
:109000005C30FFF77CF9054B24626362044BA3627A
:10901000044BE362044B236310BDC0460596000079
:109020002D960000659600009196000070B56825A9
:109030004B1E5D430E0029007431FFF7AFF9041E8B
:1090400008D000212A00016046600C30A060683220
:10905000FFF755F9200070BD836913B50400002B9C
:1090600028D18364C3640365134B144A1B6882626E
:109070000193984201D101238361200000F020F880
:109080006060200000F01CF8A060200000F018F8DC
:109090000022E06004216068FFF7A4FF012209219B
:1090A000A068FFF79FFF02221221E068FFF79AFFF6
:1090B0000123A36113BDC04630A70000D58F000077
:1090C000F8B51D4B06001D68AB69002B02D12800C6
:1090D000FFF7C2FF4835AC686B68013B05D40C2232
:1090E000A75E002F10D06834F7E72B68002B01D063
:1090F0002D68F0E704213000FFF798FF2860002872
:10910000F6D10C23336016E0012320005B42E3819B
:109110000233A38167662760A76067602761676184
:10912000A7615C3008223900FFF7E9F82000676387
:10913000A763A764E764F8BD30A70000F7B5040093
:109140000700002601914834002C16D06368A568FA
:109150000093009B013B00930DD4AB89012B08D9F0
:109160000E22AB5E013304D029003800019B9847E2
:1091700006436835EDE72468E6E73000FEBD0000F1
:10918000F0B58B8991B006000C009B0726D40E2306
:10919000C95E002904DA8023A5891D4010D10CE0A6
:1091A00001AA00F0A1FA0028F5DBF023029D1B02C2
:1091B0001D401A4BED186B425D418027FF0001E016
:1091C0000025402739003000FFF7E8F800280CD1CF
:1091D000A3899A051FD402221343A3812300473396
:1091E000236023610123636115E080220C4BB3628D
:1091F000A38920601343A38120616761002D0AD0F9
:109200000E23E15E300000F081FA002803D0012235
:10921000A3891343A38111B0F0BDC04600E0FFFF56
:10922000D58F0000C9B28218904204D003788B42D7
:1092300002D00130F8E70020704710B5884202D90B
:109240008B18984201D3002305E09B1A013A08D3FA
:10925000995C8154FAE7934203D0CC5CC454013347
:10926000F9E710BDF8B506000C001500002904D17F
:109270001100FFF793F8040018E0002A03D1FFF76C
:1092800047F82C0012E000F067FA85420ED9290059
:109290003000FFF783F8071E07D021002A00FFF7F0
:1092A00025F821003000FFF733F83C002000F8BD1E
:1092B000F0B58E6885B007000C00039201939E42C2
:1092C00043D890238A89DB001A423ED003250969DE
:1092D000236801985B1A029363695D43EB0F5D1984
:1092E000029B6D1001331B18AB4200D91D005305C2
:1092F00010D529003800FFF751F8061E14D0029A45
:109300002169FEF7F3FFA289194B13408022134312
:10931000A38112E02A003800FFF7A4FF061E0CD13B
:1093200021693800FEF7F4FF0C23402201203B6046
:10933000A38940421343A38117E0029B2661F618DC
:1093400026606561019EED1AA560019BB34200D2C3
:109350001E00320003992068FFF76FFF0020A3680A
:109360009B1BA36023689E19266005B0F0BDC04614
:109370007FFBFFFFF0B59FB0029005938B890F0034
:1093800016001B0610D50B69002B0DD14021FFF7ED
:1093900005F838603861002804D10C23029A01389E
:1093A0001360D8E040237B61002306AD6B6120335E
:1093B0006B761033AB7634002378002B03D1A31BDC
:1093C000049312D003E0252BF9D00134F4E7A31B5A
:1093D000320039000298FFF76BFF431C00D1B4E064
:1093E0006A69049B944663446B612378002B00D127
:1093F000ABE00122002352426A6002A954325218A3
:1094000001342B60EB60AB601370AB65534E217879
:1094100005223000FFF706FF002807D00123801B3C
:1094200083402A68013413432B60EFE72B68DA0688
:1094300004D55322202102A8121811701A0704D54E
:1094400053222B2102A81218117022782A2A03D045
:10945000099B00200A210EE0059A111D1268059152
:10946000002A01DB099204E05242EA60022213431F
:109470002B6001340BE02278303A092A04D84B43A0
:1094800001349B180120F6E7002800D009932378C7
:109490002E2B1ED163782A2B0AD1059B02341A1D6C
:1094A0001B680592002B01DA01235B42079310E051
:1094B00000230A201A0001346B6021783039092911
:1094C00004D84243013452180123F6E7002B00D0A0
:1094D0000792234E217803223000FFF7A3FE0028D5
:1094E00006D04023801B83402A68013413432B603D
:1094F000217806221B48661C2976FFF793FE002878
:1095000012D0194B002B06D10722059B073393433A
:109510000833059314E005AB00933A00134B290080
:10952000029800E000BF07E005AB00933A000F4B44
:1095300029000298FFF73AF90390039B013304D006
:109540006B69039A9B186B6135E7BB890B985B06C7
:1095500001D5012040421FB0F0BDC04634A7000035
:109560003AA700003EA7000000000000B1920000F2
:1095700070B504000D1E1F2D04D9162303600120B1
:1095800040421EE0426C002A04D08B00D2181368BF
:10959000002B08D1200000F031F82A000100200043
:1095A00000F01AF80DE00020012B0AD0591C03D15D
:1095B00017332360013004E000242800146098472A
:1095C000200070BD10B5034B01001868FFF7D0FFF5
:1095D00010BDC04680020020002370B5064C050077
:1095E00008001100236000F0F7F8431C03D1236842
:1095F000002B00D02B6070BDE025002010B500F0DE
:10960000DBF810BD70B50C000E25495F00F0B0F816
:10961000002803DB636D1B18636503E0A289024B1E
:109620001340A38170BDC046FFEFFFFFF8B51F00D8
:109630008B8905000C001600DB0505D50E23C95EDD
:109640000022022300F074F8A289054B2800134081
:10965000A38132000E23E15E3B0000F01FF8F8BD4D
:10966000FFEFFFFF70B50C000E25495F00F060F8BA
:10967000A389421C03D1054A1340A38104E0802240
:1096800052011343A381606570BDC046FFEFFFFF29
:1096900010B50E23C95E00F015F810BD70B50500B9
:1096A000080011000022064C22601A0000F0BAF8EF
:1096B000431C03D12368002B00D02B6070BDC04633
:1096C000E0250020002370B5064C0500080023604B
:1096D00000F062F8431C03D12368002B00D02B60FC
:1096E00070BDC046E0250020002370B5064C050083
:1096F00008001100236000F057F8431C03D12368D1
:10970000002B00D02B6070BDE0250020002370B539
:10971000064C05000800236000F056F8431C03D1F6
:109720002368002B00D02B6070BDC046E0250020D0
:1097300070B50500080011000022064C22601A00D6
:1097400000F052F8431C03D12368002B00D02B609B
:1097500070BDC046E02500200B1F1A68101F002AAC
:1097600004DA891804390B68D018043870470000EF
:1097700070B50500080011000022064C22601A0096
:1097800000F03AF8431C03D12368002B00D02B6073
:1097900070BDC046E025002058220120014B404208
:1097A0001A607047E025002058220120014B4042FA
:1097B0001A607047E025002058220120014B4042EA
:1097C0001A607047E02500205822024B00201A60E2
:1097D0007047C046E025002058220120014B40423E
:1097E0001A607047E025002058220120014B4042BA
:1097F0001A607047E025002058220120014B4042AA
:109800001A607047E0250020044A1368002B03D03B
:109810001818106018007047014BF9E7CC110020B0
:10982000E825002058220120014B40421A60704771
:10983000E0250020FEE7C046F8B5C046F8BC08BCED
:109840009E467047F8B5C046F8BC08BC9E467047B7
:1098500066616C73650074727565006C6973742061
:109860006F66202564206974656D73006F626A6598
:109870006374206F6620636C6173733A2025640003
:10988000537461636B20756E646572666C6F7700EC
:1098900036060000C8050000460600007C060000F1
:1098A000B8060000F20600002E0700005607000070
:1098B00094070000DA070000360800007C0800006A
:1098C000EA08000038090000600900009A09000059
:1098D000E40900000C0A0000440A00007E0A0000AF
:1098E000BA0A0000400B0000080C0000980C0000B1
:1098F000F60C0000400D0000620D00006A0D000033
:109900004C0E0000980E00003606000036060000DF
:1099100036060000140F00007E0F0000001000004B
:109920004A100000981000001E110000A61100004F
:10993000F41100003E12000074120000C01200007A
:109940000C13000060130000BC130000181400008A
:1099500056140000C2140000FA140000461500005E
:1099600092150000DE1500001816000064160000B5
:10997000B01600003606000036060000360600006D
:10998000201700005817000090170000BE170000B5
:10999000F617000024180000360600003606000006
:1099A00036060000360600005C180000A41800000F
:1099B0003606000036060000F01800001E190000F0
:1099C0006819000036060000360600003606000062
:1099D00096190000C6190000F6190000261A0000AA
:1099E000521A00008A1A0000B61A0000F81A000085
:1099F000221B0000521B0000821B0000AE1B000057
:109A0000DA1B00000A1C0000361C000036060000AD
:109A10003606000036060000360600003606000056
:109A2000661C0000941C0000C21C0000F01C00001A
:109A30001E1D0000561D00008E1D0000C61D0000EA
:109A4000FE1D00002C1E00005A1E00009C1E00007F
:109A50003606000036060000360600003606000016
:109A60003606000036060000360600003606000006
:109A700036060000360600003606000036060000F6
:109A80003606000036060000CA1E0000F81E000060
:109A9000070000000300000043616C6C696F706593
:109AA00000686173546F6E6500706C6179546F6EFD
:109AB0006500686173536572766F007365745365F2
:109AC00072766F0015000000010000000200000027
:109AD0000400000005000000060000000D0A564DBD
:109AE0002050616E69633A2025730D0A00496E7338
:109AF000756666696369656E74206D656D6F7279F0
:109B000020666F72204D6963726F426C6F636B7376
:109B1000206F626A656374206865617000496E73C6
:109B2000756666696369656E74206D656D6F7279BF
:109B300020666F72204D6963726F426C6F636B7346
:109B400020737461636B00626164206F626A656395
:109B50007420617420256C640A0025783A202564FD
:109B600020776F7264732C20636C61737349442097
:109B700025640A004865616465723A2025780A0008
:109B800009307825782C0A006D6973630068657860
:109B9000546F496E740073696E006E65740068617D
:109BA0007357694669007374617274576946690036
:109BB00073746F7057694669007769666953746199
:109BC000747573006D7949504164647265737300F4
:109BD0007468696E674465736372697074696F6EE7
:109BE00000636C6561725468696E67446573637283
:109BF000697074696F6E00617070656E64546F5443
:109C000068696E674465736372697074696F6E002A
:109C1000617070656E64546F5468696E6750726FDE
:109C20007065727479000D0E0F04050C0B0A06079F
:109C300008090D0E0F04050C0B0A060708096469D4
:109C400073706C6179006C696768744C6576656CDB
:109C5000006D62446973706C6179006D6244697370
:109C6000706C61794F6666006D62506C6F74006D48
:109C700062556E706C6F74006D62447261775368E8
:109C8000617065006D625368617065466F724C6506
:109C900074746572006E656F506978656C53656E9B
:109CA00064006E656F506978656C53657450696EB9
:109CB00000000000000000000100000002000000A1
:109CC0000300000004000000050000000600000082
:109CD0000700000008000000090000000A00000062
:109CE0000B0000000C0000000D0000000E00000042
:109CF0000F0000001000000012000000140000001F
:109D000016000000180000001A0000001C000000EF
:109D10001E000000200000002300000026000000BC
:109D2000290000002C0000002F000000320000007D
:109D3000360000003A0000003E0000004200000033
:109D4000460000004B0000005000000055000000DD
:109D50005A00000061000000680000006F00000071
:109D6000760000007D000000840000008B000000F1
:109D70009200000099000000A0000000A700000071
:109D8000AE000000B5000000BC000000C3000000F1
:109D9000CA000000D1000000D8000000DF00000071
:109DA000E6000000ED000000F4000000FB000000F1
:109DB000FF000000000000000008080800080A4A30
:109DC0004000000A5FEA5FEA0ED92ED36E193244D2
:109DD00089330C924C924D08080000000488080852
:109DE000040804848488000A448A4000048EC480E5
:109DF000000000048800000EC00000000008000100
:109E0000224488100C9252524C048C84848E1C8202
:109E10004C901E1EC244924C06CA525FE21FF01EB6
:109E2000C13E02448ED12E1FE24488100ED12ED1A5
:109E30002E0ED12EC488000800080000048004887B
:109E40000244880482000EC00EC008048244880EBA
:109E5000D126C0040ED135B36C0C925ED2521C9246
:109E60005C925C0ED010100E1C9252525C1ED01CE4
:109E7000901E1ED01C90100ED013712E12525ED266
:109E8000521C8808081C1FE242524C12549814922B
:109E9000101010101E113B75B131113935B3710C12
:109EA0009252524C1C925C90100C92524C861C9216
:109EB0005C92510ED00C825C1FE484848412525256
:109EC000524C1131312A44113135BB7112524C922E
:109ED00052112A4484841EC488101E0EC808080E1D
:109EE00010080482410EC242424E048A4000000023
:109EF0000000001F0804800000000ED2524F101016
:109F00001C925C000ED0100E02424ED24E0C925C9F
:109F1000900E06C81C88080ED24EC24C10101C921F
:109F2000520800080808024002424C10149814928B
:109F30000808080806001B75B131001C9252520037
:109F40000C92524C001C925C90000ED24EC2000E3D
:109F5000D010100006C8049808080EC80700125256
:109F6000524F0011312A4400113135BB00124C8C84
:109F70009200112A4498001EC4881E06C48C848650
:109F8000080808080818080C881800000C836025C9
:109F9000642025642025642025640A00436F6D70C9
:109FA000616374656420466C61736820636F6465E7
:109FB0002073746F72650A2564206279746573205A
:109FC0007573656420282564252529206F66202562
:109FD00064002564202564202564202825642077DA
:109FE0006F72647329002564207265636F726473F5
:109FF0002C20256420776F7264732C206D61784962
:10A00000442025642C20636F6D70616374696F6EEA
:10A01000206379636C65732025640042616420725B
:10A0200065636F726420666F756E64206475726913
:10A030006E6720696E697469616C697A6174696FB1
:10A040006E210A004E6F7420656E6F75676820720E
:10A050006F6F6D206576656E206166746572206332
:10A060006F6D70616374696F6E0A00526573746F0F
:10A070007265642025642073637269707473005381
:10A0800074617274656400536372697074732063E1
:10A090006C6561726564002D2D2D2D2D0A005065B3
:10A0A0007273697374656E74204D656D6F7279207B
:10A0B000546573740A0A000A496E697469616C69AF
:10A0C0007A696E67204D656D6F72790A004D656D16
:10A0D0006F727920696E74697469616C697A6564FC
:10A0E0003B2077726974696E67207265636F726472
:10A0F000732E2E2E0A005265636F726420617420E5
:10A100006F66667365742025643A20256420256493
:10A110002025642025642028256420776F726473CD
:10A12000290A0046696E616C3A2063757272656E29
:10A1300074202564207573656420256420633020B5
:10A1400025642063312025640A006E6F6E650072FD
:10A150006164696F0064697361626C65526164690E
:10A160006F006D65737361676552656365697665D8
:10A1700064007061636B6574526563656976650040
:10A180007061636B657453656E64007265636569C5
:10A19000766564496E7465676572007265636569AA
:10A1A0007665644D65737361676554797065007297
:10A1B00065636569766564537472696E670073657B
:10A1C0006E64496E74656765720073656E64506194
:10A1D00069720073656E64537472696E67007365AB
:10A1E000744368616E6E656C0073657447726F7559
:10A1F0007000736574506F776572007369676E6184
:10A200006C537472656E677468004E6F2066726579
:10A2100065207461736B20656E7472696573004D9F
:10A22000656D6F727920636C656172656400416C65
:10A230006C207461736B732073746F70706564004D
:10A2400076303633002025732025730073656E73D6
:10A250006F72730074656D706572617475726500FC
:10A2600074696C74580074696C74590074696C7406
:10A270005A00746F75636852656164006932635295
:10A28000656164006932635772697465007466744D
:10A2900000656E61626C65446973706C617900730E
:10A2A0006574506978656C006C696E6500726563F1
:10A2B0007400726F756E64656452656374006369DF
:10A2C00072636C6500747269616E676C65007465B9
:10A2D000787400746674546F75636865640074669E
:10A2E00074546F7563685800746674546F7563684E
:10A2F0005900746674546F75636850726573737532
:10A3000072650057656C636F6D6520746F204D69D1
:10A3100063726F426C6F636B732100535049436CDF
:10A320006173733A3A535049436C617373284E52C8
:10A33000465F5350495F547970652A2C2075696EC9
:10A3400074385F742C2075696E74385F742C2075B6
:10A35000696E74385F742900705F73706920213DE5
:10A36000204E554C4C002F55736572732F6A6F68E1
:10A370006E6D616C6F6E65792F4C69627261727976
:10A380002F41726475696E6F31352F7061636B6137
:10A390006765732F73616E646565706D6973747240
:10A3A000792F68617264776172652F6E5246352F1E
:10A3B000302E362E302F6C69627261726965732F90
:10A3C0005350492F5350492E637070000000000015
:10A3D0000000000063460000294600004F460000D0
:10A3E00059460000894600004D460000000000006C
:10A3F0000100000002000000160000000400000040
:10A400000500000006000000070000000800000032
:10A41000090000000A0000000B0000000C00000012
:10A420000D0000000E0000000F0000001A000000E8
:10A430001B000000140000001300000011000000C9
:10A4400003000000100000001C0000001D000000C0
:10A450001E000000120000001500000017000000A0
:10A460001800000019000000FB21F93FFB21094002
:10A470007CD91240FB2119407A6A1F407CD92240C6
:10A48000BBFD2540FB2129403A462C407A6A2F40EB
:10A490005C4731407CD932409C6B3440BBFD354039
:10A4A000DB8F3740FB2139401BB43A403A463C40F1
:10A4B0005AD83D407A6A3F404C7E40405C4741401C
:10A4C0006C1042407CD942408CA243409C6B44407B
:10A4D000AC344540BBFD4540CBC64640DB8F4740D2
:10A4E000EB584840FB21494083F9A200444E6E00DE
:10A4F000FC291500D1572700DD34F50062DBC000D0
:10A500003C999500419043006351FE00BBDEAB00D7
:10A51000B761C5003A6E2400D24D42004906E00002
:10A5200009EA2E001C92D100EB1DFE0029B11C008F
:10A53000E83EA700F535820044BB2E009CE984006C
:10A54000B4267000417E5F00D691390053833900F4
:10A550009CF439008B5F840028F9BD00F81F3B0094
:10A56000DEFF97000F980500112FEF000A5A8B00AD
:10A570006D1F6D00CF7E360009CB2700464FB70018
:10A580009E663F002DEA5F00BA277500E5EBC70025
:10A590003D7BF100F739070092528A00FB6BEA001D
:10A5A0001FB15F00085D8D00300356007BFC460044
:10A5B000F0AB6B0020BCCF0036F49A00E3A91D007D
:10A5C0005E619100081BE60085996500A0145F009C
:10A5D0008D40680080D8FF0027734D0006063100CB
:10A5E000CA561500C9A873007BE260006B8CC000DE
:10A5F000020000000300000004000000060000004C
:10A6000000000040FB21F93F000000002D44743E93
:10A61000000000809846F83C0000006051CC783B78
:10A6200000000080831BF0390000004020257A38AC
:10A63000000000802282E336000000001DF369352F
:10A640000000000000000000215E0000115C00001E
:10A65000915E0000A55E00009B5E00001D5E000094
:10A66000115E0000B15E00003D5E00000D5E000066
:10A670006C6A0000CA690000CA690000C86900006D
:10A680005E6A00005E6A0000546A0000C86900004B
:10A690005E6A0000546A00005E6A0000C86900003B
:10A6A000646A0000646A0000646A0000EE6A0000E8
:10A6B0006C7600002C7500002C7500002A750000D7
:10A6C0004476000044760000367600002A750000CB
:10A6D0004476000036760000447600002A750000BB
:10A6E0004C7600004C7600004C7600004C78000060
:10A6F0002C2066756E6374696F6E3A200061737307
:10A70000657274696F6E2022257322206661696C00
:10A7100065643A2066696C6520222573222C206CC2
:10A72000696E65202564257325730A0043000000C7
:10A7300020020020232D302B2000686C4C00656621
:10A740006745464700303132333435363738394182
:10A750004243444546003031323334353637383998
:10A760006162636465660000202020202020202094
:10A7700020282828282820202020202020202020B1
:10A7800020202020202020208810101010101010D1
:10A790001010101010101010040404040404040419
:10A7A00004041010101010101041414141414101AA
:10A7B0000101010101010101010101010101010189
:10A7C0000101011010101010104242424242420298
:10A7D0000202020202020202020202020202020259
:10A7E0000202021010101020000000000000000003
:10A7F0000000000000000000000000000000000059
:10A800000000000000000000000000000000000048
:10A810000000000000000000000000000000000038
:10A820000000000000000000000000000000000028
:10A830000000000000000000000000000000000018
:10A840000000000000000000000000000000000008
:10A8500000000000000000000000000000000000F8
:10A8600000000000000000000000000000000000E8
:10A8700000000000000000000000000000000000D8
:10A8800000000000000000000000000000000000C8
:10A8900000000000000000000000000000000000B8
:10A8A00000000000000000000000000000000000A8
:10A8B0000000000000000000000000000000000098
:0CA8C0000000000000000000000000008C
:08A8CC00A858FF7F0100000005
:10A8D400FFFFFFFF40060000A19A0000D91F0000FF
:10A8E400A99A0000D51F0000B29A0000DD1F0000E5
:10A8F400BB9A0000E11F00008D9B00002124000092
:10A90400969B0000752400009E9B000051250000CA
:10A91400A69B000081250000B09B00009525000047
:10A92400B99B00009F250000C49B00008B250000FC
:10A93400D09B00005F250000E19B0000752500000E
:10A94400F79B000069250000109C000055250000BD
:10A95400469C0000C5250000519C0000792A000097
:10A964005B9C00000D280000689C00002D2800005E
:10A974006F9C00007D280000789C0000CD2800001A
:10A98400849C0000A52A0000959C0000B5290000C5
:10A99400A29C0000952600001800000055A10000AC
:10A9A400D934000062A10000DD34000072A100006F
:10A9B400E134000080A10000E53400008BA1000018
:10A9C400A13400009BA10000B5340000AFA1000039
:10A9D400A5340000BEA10000E9340000CAA10000B3
:10A9E400ED340000D3A10000F1340000DEA100002A
:10A9F400F5340000E9A10000D5340000F2A1000004
:10AA04009D340000FBA10000AD34000054A20000FE
:10AA14003D43000060A200005743000066A200000E
:10AA2400874300006CA200000B43000072A20000E8
:10AA3400C54000007CA20000B943000084A20000CD
:10AA4400F141000091A20000454400009FA20000D3
:10AA540049440000A8A200004D440000ADA200003B
:10AA640051440000B2A2000055440000BEA2000000
:10AA740059440000C5A200005D440000CEA20000BD
:10AA840061440000D3A2000065440000DEA200007F
:10AA940069440000E8A2000041440000F2A2000062
:10AAA4003D44000003000000020000000800000014
:10AAB4000A000000FFFFFFFF00000000010000008B
:10AAC4000000020001000000FFFFFFFF0000000083
:10AAD400020000000000040002000000FFFFFFFF6E
:10AAE4000000000003000000000008000300000054
:10AAF4000000000068A8000088A80000A8A80000C2
:10AB04000000000000000000000000000000000041
:10AB14002CA700000000000000000000000000005E
:10AB24000000000000000000000000000000000021
:10AB34000000000000000000000000000000000011
:10AB44000000000000000000000000000000000001
:10AB54002002002067A7000039010000F945000029
:10AB640019490000156100000D01000000000000FB
:0400000300005CE1BC
:00000001FF
